:1000000016C3000033C3000031C300002FC300003B
:100010002DC300002BC3000029C3000027C300002C
:1000200025C3000023C3000021C300001FC300003C
:100030000C94903B1BC3000019C3000017C30000C1
:1000400015C3000013C300000C947C3B0FC30000D9
:100050000DC300000BC3000009C3000007C300006C
:1000600005C3000003C3000001C30000FFC200007D
:10007000FDC20000FBC20000F9C20000F7C2000090
:10008000F5C20000F3C20000F1C20000180A1D0A08
:100090002B0A300A350A3A0A3F0A440AD20DD70D14
:1000A000E50DEA0DEF0DF40DF90DFE0D32123512CE
:1000B00038123B123E12411244124712C01DE41D79
:1000C000F71D071E0A1E1A1E2A1E431ED51DD81D07
:1000D0003A1E3D1E401EDB1DDE1DE11D3123472360
:1000E0005B23732389239F23C323D923EF23B925BC
:1000F000102606275D2753285529172AE92AEA2BB7
:10010000252C792CBA2CC32C132D632D662D692D2B
:100110006C2D6F2D722D752D782D223038304E308C
:1001200065307B309130A730BD301131143117313B
:100130001A311D312031233126317E31FA317632A8
:10014000FF328833FF337B34F7347335EC3559365F
:10015000D0365637D93700000000000000000404F4
:100160000404000400000A0A0A00000000000A0A51
:100170001F0A1F0A0A00040F140E051E0400181996
:100180000204081303000C12140814120D000C04CE
:100190000800000000000204080808040200080427
:1001A0000202020408000004150E150400000004F9
:1001B000041F04040000000000000C0408000000FC
:1001C000001F0000000000000000000C0C000001F7
:1001D0000204081000000E11131519110E00040C72
:1001E000040404040E000E11010204081F001F0283
:1001F000040201110E0002060A121F0202001F1063
:100200001E0101110E000608101E11110E001F0123
:100210000204080808000E11110E11110E000E1133
:10022000110F01020C000001020408100000000C74
:100230000C000C040800020408100804020000006E
:100240001F001F00000008040201020408000E1134
:100250000102040004000E11010D15150E000E110F
:1002600011111F1111001E11111E11111E000E116E
:10027000101010110E001C12111111121C001F1071
:10028000101E10101F001F10101E101010000E1155
:10029000101711110E001111111F111111000E0470
:1002A000040404040E000702020202120C001112E0
:1002B0001418141211001010101010101F00111B30
:1002C00015151111110011111915131111000E112D
:1002D000111111110E001E11111E101010000E111F
:1002E000111115120D001E11111E141211000F1004
:1002F000100E01011E001F04040404040400111167
:10030000111111110E0011111111110A0400111116
:10031000111115150E0011110A040A111100111105
:10032000110A040404001F01020408101F000E0833
:10033000080808080E00110A1F041F0404000E021A
:10034000020202020E00040A110000000000000078
:10035000000000001F000804000000000000000072
:100360000E010F110F0010101E1111111E000000C0
:100370000E1010110E0001010D1311110F000000DD
:100380000E111F100E000609081C08080800000FB7
:1003900011110F010E001010161911111100040097
:1003A0000C0404040E000200060202120C001010DD
:1003B0001214181412001808080808081C0000007D
:1003C0001A15151111000000161911111100000065
:1003D0000E1111110E0000001E111E101000000061
:1003E0000F110F010100000016191010100000007D
:1003F0000E100E011E0008081C0808090600000067
:10040000111111130D0000001111110A0400000058
:10041000111111150A000000110A040A1100000050
:1004200011110F010E0000001F0204081F003844C4
:1004300044447C4444007C40407844447800784400
:100440004478444478007C404040404040000C14D4
:10045000242424243C447C40407840407C00545474
:100460005438545454003844041804443800444464
:100470004C546444440054444C5464444400444840
:100480005060504844001C24242424246400446CFC
:100490005454444444004444447C44444400384458
:1004A0004444444438007C44444444444400784434
:1004B00044784040400038444040404438007C107C
:1004C0001010101010004444443C044438003854C8
:1004D0005454381010004444281028444400444424
:1004E000444444447E02444444443C040400545480
:1004F000545454547C005454545454547E02602038
:100500002038242438004444446454546400404057
:100510004078444478003844041C0444380048546B
:100520005474545448003C44443C14244400000097
:1005300038043C443C0000007840784478000000D7
:10054000784C784C78000000784040404000000033
:10055000182828287C44000038447C403C000000D7
:1005600054543854540000007804380478000000D3
:10057000444C546444000010444C54644400000053
:1005800044487048440000001C24444444000000D7
:10059000446C545444000000484878484800000027
:1005A0003844444438000000784848484800000077
:1005B0007048704040000000384040403800000063
:1005C0007C1010101000000048483808700000002F
:1005D000385454381000000044281028440000000B
:1005E000484848487C040000484838080800000093
:1005F000545454547C000000545454547E0200005F
:1006000060203C223C0000004242724A720000001E
:1006100040407844780000007008780870000000BE
:100620004C5272524C0000003C443C4444001124A3
:100630001FBECFEFD0E1DEBFCDBF15E0A0E0B1E03F
:10064000E6E7F4E800E00BBF02C007900D92A43D7E
:10065000B107D9F726E0A4EDB5E001C01D92A63898
:10066000B207E1F70E94EE3B0C943942C9CCE2E6B6
:10067000F0E090819E7F9083908194609083908140
:10068000977F9083A8988BBB8DE08A95F1F7000047
:10069000A89A8081886080830895E2E6F0E09081E6
:1006A000916090839081946090839081977F9083F4
:1006B000A8988BBB8DE08A95F1F70000A89A8081FD
:1006C000886080830895CF93C82F892FE6DF8C2F11
:1006D000CF91E3CFE2E6F0E020812160208320810A
:1006E000246020832081277F2083A8988BBB92BB26
:1006F0008DE08A95F1F70000A89A80818860808358
:100700000895CF93C82F86E3B2DFC13049F030F0AF
:10071000C23041F0C33059F488EE07C088E403C00A
:1007200088E203C088E8B9DF04C0B7DF0BC0CD7F23
:1007300049F48FEE90E09093D7058093D6058FE330
:1007400091E008C08FE391E09093D7058093D605A0
:100750008FEE90E09093D5058093D405CF910895C6
:10076000CF93C82F8FEF8ABB81BB8093610081E05C
:1007700084BBE2E6F0E080818260808381E077DF05
:100780002FEF89E698E1215080409040E1F700C0CA
:10079000000080EC6CDF85E280DF81EC68DF81E1C6
:1007A0007CDF85EC64DF8BE278DF8BE276DF87EC41
:1007B0005EDF86E872DF8C2FA4DF8AE358DF85E0F6
:1007C0006CDF81EB54DF80E068DF88E166DF86EB79
:1007D0004EDF8AE062DF82E860DF87E25EDF81E190
:1007E00046DF2FEF8DEE92E0215080409040E1F700
:1007F00000C0000089E2CF913ACF0F931F93CF93AF
:10080000DF938C01EB018AE232DFC8015CDFCE01AD
:10081000DF91CF911F910F9156CF0F931F93CF93DD
:10082000DF938C01EB018BE222DFC8014CDFCE01AC
:10083000DF91CF911F910F9146CFCF93DF93EB01C3
:10084000BC01DBDFBE01CE01E8DF8CE2DF91CF919E
:100850000ECFCF93DF93EA01F0DFCE01DF91CF918E
:1008600039CF8F929F92AF92BF92CF92DF92EF9249
:10087000FF920F931F93CF93DF93A8956817790783
:1008800038F4862797276827792786279727A895FA
:100890002417350738F442275327242735274227C2
:1008A0005327A895A091D605B091D705FC01A817AC
:1008B000B90708F4FD016B01A617B70708F46D012D
:1008C0008091D4059091D505EA018417950708F425
:1008D000EC0179018217930708F47C01A895960131
:1008E0002F5F3F4F2E1B3F0BD7011196AC1BBD0B4B
:1008F0000E94013F4B015C01B601CF017EDFA8954C
:10090000B701CE018ADF8CE2B2DEA895C12CD12CD2
:100910007601C814D904EA04FB0449F0C801DADE00
:10092000A8958FEFC81AD80AE80AF80AF2CFDF9123
:10093000CF911F910F91FF90EF90DF90CF90BF90DC
:10094000AF909F908F9008950F931F93411551057D
:1009500079F02115310561F0FA01AB01615071099F
:10096000260F371FBC01615071096E0F7F1F79DFA1
:100970001F910F9108952F923F924F925F926F9225
:100980007F928F929F92AF92BF92CF92DF92EF921F
:10099000FF920F931F93CF93DF93CDB7DEB7679787
:1009A0000FB6F894DEBF0FBECDBF5C01798B688BAC
:1009B000598748873B872A870F83F12C28E0029FBD
:1009C000C00111241A821982E8E0F0E0FF8BEE8B5F
:1009D00047019C01285F31093B8B2A8BFC01E052C7
:1009E000F340FD8BEC8BC888D98889819A81C80E29
:1009F000D91E8A899B89EE89FF898E1B9F0B9C01DA
:100A00002A5A3E4F3F872E878C899D898E1B9F0BCC
:100A1000FC01EA5AFE4FFD87EC871E821D821C8274
:100A20001B8287E0682E712C412C512C212C312CFB
:100A3000FF81F7FD1EC0EE85FF85849190E0062CB6
:100A400002C0959587950A94E2F780FF08C0088553
:100A500019859701A701B6018D819E8107C00A857E
:100A60001B859701A701B6018B819C818A0D9B1D77
:100A700020C0FF81F03CF0F0EC85FD85849190E092
:100A8000062C02C0959587950A94E2F780FF09C06D
:100A9000088519859701A701B601C501820D931D2F
:100AA00008C00A851B859701A701B601C501840D01
:100AB000951D4ADF280C391C480C591CF1E06F1AAF
:100AC00071082B813C81280D391D3C832B838D813E
:100AD0009E81880D991D9E838D839FEF69167906EF
:100AE00009F0A6CFEE89FF893197FF8BEE8B298124
:100AF0003A812E0D3F1D3A832983EF2B09F073CFE6
:100B000067960FB6F894DEBF0FBECDBFDF91CF91D1
:100B10001F910F91FF90EF90DF90CF90BF90AF901B
:100B20009F908F907F906F905F904F903F902F900D
:100B300008954F925F926F927F928F929F92AF92A1
:100B4000BF92CF92DF92EF92FF920F931F93CF93BA
:100B5000DF93EC016B014A013901102F88E0089FF7
:100B6000500111242701F20101912F010023B1F05E
:100B70002091D6053091D705CE0108962817390760
:100B800020F4CA0CDB1CC1E0D0E0E12E9301A401EB
:100B9000B601CE01F0DECA0DDB1DE5CFDF91CF91AE
:100BA0001F910F91FF90EF90DF90CF90BF90AF908B
:100BB0009F908F907F906F905F904F9008956F926D
:100BC0007F928F929F92AF92BF92CF92DF92EF92DD
:100BD000FF920F93CF93DF9300D000D0CDB7DEB755
:100BE0006C015B014A013901C70119821A821B821B
:100BF0001C824AE0BE016F5F7F4F0E94103FCE0112
:100C000001967C019301A401B501C60192DF0F900A
:100C10000F900F900F90DF91CF910F91FF90EF9079
:100C2000DF90CF90BF90AF909F908F907F906F900C
:100C300008950F931F932091D4053091D5056091AD
:100C4000D6057091D7058C0140E050E080E090E03F
:100C500008DE1F910F910895EF92FF920F931F935B
:100C6000CF93DF93EB018A017901BC01640F751FFB
:100C7000C4DDBE01CE01D1DD8CE2F9DCC0E0D0E004
:100C8000C017D10721F0C70125DD2196F9CFDF91EB
:100C9000CF911F910F91FF90EF900895EF92FF92E7
:100CA0000F931F93CF93DF93EB018A017901BC016E
:100CB000A4DDBE01600F711FCE01AFDD8CE2D7DC79
:100CC000C0E0D0E0C017D10721F0C70103DD2196B5
:100CD000F9CFDF91CF911F910F91FF90EF90089581
:100CE0002F923F924F925F926F927F928F929F923C
:100CF000AF92BF92CF92DF92EF92FF920F931F932A
:100D0000CF93DF9300D000D000D0CDB7DEB76C0119
:100D10007B015A0139012801261B370B3A832983AD
:100D20008A01081B190B17FF03C0119501951109C2
:100D3000CA14DB0420F022242A94322C03C022247B
:100D40002394312C89819A819E838D8397FF05C0DE
:100D50009195819591099E838D832D813E81319559
:100D6000219531093C832B83E614F70428F08FEF9B
:100D70009FEF9A83898304C021E030E03A8329837E
:100D800048018D819E81881A990AA201B701C60186
:100D900060DDC401880F991F2B813C818217930766
:100DA00064F0CA14DB0499F02D813E81821A930A03
:100DB000C20CD31C0817190744F3E614F70439F0E2
:100DC000800E911E89819A81E80EF91EDECF26964B
:100DD0000FB6F894DEBF0FBECDBFDF91CF911F914C
:100DE0000F91FF90EF90DF90CF90BF90AF909F90CA
:100DF0008F907F906F905F904F903F902F900895CD
:100E0000AF92BF92CF92DF92EF92FF920F931F9318
:100E1000CF93DF937C016B01EA01590198011CDF3C
:100E2000B501615071096C0D7D1D9801AE01C701BE
:100E300013DF9801A501B601C70130DFCE0101978C
:100E40009801A501B6018E0D9F1DDF91CF911F91D5
:100E50000F91FF90EF90DF90CF90BF90AF901ECF9B
:100E60002F923F924F925F926F927F928F929F92BA
:100E7000AF92BF92CF92DF92EF92FF920F931F93A8
:100E8000CF93DF931C012B01690150E0002711274C
:100E9000041B150BC1E0D0E0C41BD50BCC0FDD1F2C
:100EA000E12CF12CA6015701A40CB51CB5013101B0
:100EB000601A710AC301CDDCA601B5014801820C9C
:100EC000931CC401C6DCA6015201AE18BF08B501CF
:100ED000C401BFDCA601B501C301BBDCEC16FD06F5
:100EE000B4F08FEFE81AF80AC701880F991F01962E
:100EF0008C0F9D1F22273327201B310BE216F30690
:100F000039F40C171D074CF0C0E0D0E001C0CE0151
:100F10000C171D0714F0EC01C5CF0F5F1F4F980190
:100F2000220F331F2F5F3F4F820F931F10161106A2
:100F300094F7DF91CF911F910F91FF90EF90DF9089
:100F4000CF90BF90AF909F908F907F906F905F9069
:100F50004F903F902F9008954F925F926F927F92A3
:100F60008F929F92AF92BF92CF92DF92EF92FF92B9
:100F70000F931F93CF93DF93EC015B014A0139017B
:100F800028018601ADDE9701A201B301C401A8DEEC
:100F90009501AE01B701C201A3DEDF91CF911F9190
:100FA0000F91FF90EF90DF90CF90BF90AF909F9008
:100FB0008F907F906F905F904F900895CF93C82F40
:100FC0008A3011F48DE0FADF5D9BFECFCCB980E072
:100FD00090E0CF910895CF92DF92EF92FF920F931E
:100FE0001F93A8950FEF1FEF21E430E04FE550E08D
:100FF00065E070E085E090E003DFA89521E430E053
:101000004FE550E06BE470E085E090E0F9DE2BE422
:1010100030E04FE550E061E970E085E090E0F0DE1F
:10102000A2E2EA2EA5E0FA2E01E02FE130E04FEF38
:101030005FEF60E570E082E190E07BDDBDE1EB2EEB
:10104000B5E0FB2E2FE130E04FEF5FEF6AE570E097
:1010500083E290E06EDD0FEF1FEF21E430E04FE51B
:1010600050E065E070E08CED90E0CADE21E430E015
:101070004FE550E06BE470E08CED90E0C1DE2BE4D6
:1010800030E04FE550E061E970E08CED90E0B8DED3
:1010900012E2E12E15E0F12E01E02FE130E04FEFFA
:1010A0005FEF60E570E08BEE90E043DD87E1E82ED6
:1010B00085E0F82E2FE130E04FEF5FEF6AE570E05A
:1010C0008CEF90E036DD99E4E92E92E0F92E2FE1E5
:1010D00030E04FEF5FEF66EE70E08AE090E029DDF0
:1010E000A8958091100690911106019709F04FC0C4
:1010F0000FE110E024E430E048E550E064E970E0FE
:1011000088E090E021DC2CE430E04EE650E06CE832
:1011100070E089E690E018DC24E430E048E550E037
:1011200064E970E080EE90E00FDC20EE37E048E20A
:1011300064EB70E080EA90E093DE20EE37E047E277
:1011400064EB70E080EA90E08BDE20EE37E04BE26B
:1011500064EB70E080EA90E083DE20EE37E045E269
:1011600064EB70E080EA90E07BDEE0EECE2EE7E01C
:10117000DE2EF4EBEF2EF12C07EB10E028EC30E044
:1011800044E950E060EA70E084E990E0E5DEA8958B
:101190008091100690911106892B09F051C00FE142
:1011A00010E024E430E048E550E064E970E088E0D5
:1011B00090E0CADB2CE430E04EE650E06CE870E0F2
:1011C00089E690E0C1DB24E430E048E550E064E9E2
:1011D00070E080EE90E0B8DB20E038EF48E264EBAE
:1011E00070E080EA90E03CDE20E038EF47E264EB1C
:1011F00070E080EA90E034DE20E038EF4BE264EB10
:1012000070E080EA90E02CDE20E038EF45E264EB0D
:1012100070E080EA90E024DE00E018EF23E230E0A6
:1012200045E050E065EA70E086E990E08DDB23E27E
:1012300030E045E050E065EA70E085EA90E084DB6C
:10124000A8958091120690911306892B79F4A895A0
:101250007DE0E72E75E0F72E01E02FE130E04FEF63
:101260005FEF63E270E08AE090E063DC8091120659
:10127000909113060197E1F4A89556ECE52E55E000
:10128000F52E01E02FE130E04FEF5FEF64E170E019
:1012900084E190E04EDC60ECE62E65E0F62E2FE176
:1012A00030E04FEF5FEF68E270E08EE190E041DC0C
:1012B000A89580911206909113060297E1F4A895E3
:1012C00039EBE32E35E0F32E01E02FE130E04FEF74
:1012D0005FEF64E170E084E190E02BDC40ECE42E11
:1012E00045E0F42E2FE130E04FEF5FEF68E270E071
:1012F0008EE190E01EDCA895809112069091130675
:10130000039779F4A89522EBE22E25E0F22E01E076
:101310002FE130E04FEF5FEF63E270E089E190E0B2
:1013200008DCA8958091120690911306049779F431
:10133000A89593EDE92E94E0F92E01E02FE130E03D
:101340004FEF5FEF63E270E08FE090E0F2DBA89593
:1013500080911206909113060597E1F4A8950DEC83
:10136000E02E04E0F02E01E02FE130E04FEF5FEFE0
:1013700064E170E089E190E0DCDB83ECE82E84E05E
:10138000F82E2FE130E04FEF5FEF63E270E08FE087
:1013900090E0CFDBA89580911206909113060697F6
:1013A000E1F4A895BDECEB2EB4E0FB2E01E02FE1BB
:1013B00030E04FEF5FEF64E170E089E190E0B9DB8E
:1013C00011EBE12E14E0F12E2FE130E04FEF5FEF53
:1013D00063E270E08FE190E0ACDBA89580911206AB
:1013E00090911306079779F4A895A8E9EA2EA4E04E
:1013F000FA2E01E02FE130E04FEF5FEF63E270E0A3
:101400008FE090E096DB8091120690911306892B75
:1014100009F048C0A895E09171068E2F90E08830C1
:10142000910508F03FC0FC01EA5BFF4F0C94F83EC9
:10143000F3E9EF2EF4E0FF2E04C0EEE8EE2EE4E038
:10144000FE2E02E02FE130E04FEF5FEF6EE170E043
:101450008BEE90E026C074E8E72E74E0F72E18C0FB
:101460006AE7E62E64E0F62E13C050E7E52E54E05E
:10147000F52E0EC046E6E42E44E0F42E09C03CE50D
:10148000E32E34E0F32E04C022E5E22E24E0F22E17
:1014900001E02FE130E04FEF5FEF6EE170E086EEAC
:1014A00090E047DB8091120690911306019701F5B9
:1014B000A89580911B06813069F038F08230C1F424
:1014C00000E7E02E04E0F02E09C094E8E92E94E055
:1014D000F92E04C08AE7E82E84E0F82E01E02FE11F
:1014E00030E04FEF5FEF6EE170E086EE90E021DBE1
:1014F0008091120690911306029701F5A8958091AC
:101500002206813069F038F08230C1F4A0E7EA2E7B
:10151000A4E0FA2E09C014E8E12E14E0F12E04C074
:10152000BAE7EB2EB4E0FB2E01E02FE130E04FEF05
:101530005FEF6EE170E086EE90E0FBDA80911206DC
:1015400090911306039779F4A895FEEDEF2EF4E041
:10155000FF2E01E02FE130E04FEF5FEF6EE170E032
:101560008EEE90E0E6DA80911206909113060497D1
:1015700001F5A89580917C06813069F038F08230C1
:10158000C1F460E7E62E64E0F62E09C0E4E8EE2E32
:10159000E4E0FE2E04C07AE7E72E74E0F72E01E0C7
:1015A0002FE130E04FEF5FEF6EE170E086EE90E00C
:1015B000C0DA8091120690911306059701F5A8955F
:1015C00080917006813069F038F08230C1F430E7E4
:1015D000E32E34E0F32E09C054E8E52E54E0F52E56
:1015E00004C04AE7E42E44E0F42E01E02FE130E0AD
:1015F0004FEF5FEF6EE170E086EE90E09ADA809157
:10160000120690911306069701F5A89580916D0634
:10161000813069F038F08230C1F480E7E82E84E050
:10162000F82E09C024E8E22E24E0F22E04C09AE746
:10163000E92E94E0F92E01E02FE130E04FEF5FEF6B
:101640006EE170E086EE90E074DA8091120690917F
:101650001306079709F4A8951F910F91FF90EF903B
:10166000DF90CF900895CF92DF92EF92FF920F9389
:101670001F93A89500EE17E021E430E048EC50E01D
:101680006AEA70E085E090E05FD90FEF1FEF21E498
:1016900030E048EC50E063E270E085E090E0B0DBE1
:1016A00086E6E82E82E0F82E01E02FE130E040EE01
:1016B00057E06CE370E088E290E03BDA0FEF1FEF59
:1016C00020E530E040E550E065E070E08BEE90E032
:1016D00097DB90EEC92E97E0D92E24E1E22EF12C73
:1016E00003E111E026E430E041E351E066E470E01C
:1016F00085EF90E031DC37E1E32EF12C24E430E09B
:101700004FE251E064E470E087EF90E025DC0FEFFA
:101710001FEF20E530E040E550E064E670E08BEE3E
:1017200090E06EDB45EAE42EF12C03E111E023E7C3
:1017300030E041E351E063E770E085EF90E00CDCDE
:1017400053EAE52EF12C25E730E04FE251E065E762
:1017500070E087EF90E000DC65E3E62E65E0F62EB2
:1017600002E020EE37E040E050E068EC70E08DE20F
:1017700090E0DFD91F910F91FF90EF90DF90CF9015
:101780000895CF92DF92EF92FF920F931F93A89547
:1017900000EE17E021E430E048EC50E06AEA70E047
:1017A00085E090E0D1D80FEF1FEF21E430E048EC66
:1017B00050E063E270E085E090E022DB82EAE82E10
:1017C00084E0F82E01E02FE130E040EE57E06CE3DA
:1017D00070E088E290E0ADD90FEF1FEF20E530E038
:1017E00040E550E065E070E08BEE90E009DB90EEC4
:1017F000C92E97E0D92E24E1E22EF12C03E111E06D
:1018000026E430E041E351E066E470E085EF90E0EB
:10181000A3DB37E1E32EF12C24E430E04FE251E08A
:1018200064E470E087EF90E097DB0FEF1FEF20E5B7
:1018300030E040E550E064E670E08BEE90E0E0DA06
:1018400045EAE42EF12C03E111E023E730E041E327
:1018500051E063E770E085EF90E07EDB53EAE52E30
:10186000F12C25E730E04FE251E065E770E087EFCB
:1018700090E072DB6EECE62E65E0F62E02E020EEE4
:1018800037E040E050E068EC70E08DE290E051D944
:101890001F910F91FF90EF90DF90CF900895CF921E
:1018A000DF92EF92FF920F931F93A89500EE17E03F
:1018B00021E430E048EC50E06AEA70E085E090E036
:1018C00043D80FEF1FEF21E430E048EC50E063E233
:1018D00070E085E090E094DA81E4E82E84E0F82E70
:1018E00001E02FE130E040EE57E06CE370E088E289
:1018F00090E01FD90FEF1FEF20E530E040E550E00A
:1019000065E070E08BEE90E07BDA90EEC92E97E018
:10191000D92E24E1E22EF12C03E111E026E430E09F
:1019200041E351E066E470E085EF90E015DB37E1DC
:10193000E32EF12C24E430E04FE251E064E470E067
:1019400087EF90E009DB0FEF1FEF20E530E040E587
:1019500050E064E670E08BEE90E052DA45EAE42E67
:10196000F12C03E111E023E730E041E351E063E7CC
:1019700070E085EF90E0F0DA53EAE52EF12C25E7F0
:1019800030E04FE251E065E770E087EF90E0E4DAA5
:1019900066E4E62E65E0F62E02E020EE37E040E059
:1019A00050E068EC70E08DE290E0C3D81F910F9199
:1019B000FF90EF90DF90CF900895CF93DF9300D00A
:1019C00000D0CDB7DEB7809163001C821B821A82E3
:1019D0001982BE016F5F7F4FCE0103960E945B3D6F
:1019E0008B819C81853C994068F089819A81843AF9
:1019F000964040F489819A818D32914018F082E0BE
:101A000080933A068B819C81803D974090F48B8136
:101A10009C818139914068F089819A81843A96400D
:101A200040F489819A818D32914018F083E080934F
:101A30003A068B819C818032934068F489819A8137
:101A400084379E4040F489819A81813D974018F007
:101A500081E080933A068B819C81843C994060F4BC
:101A60008B819C81893E934038F089819A81813DA8
:101A7000974010F010923A0680913A060F900F901E
:101A80000F900F90DF91CF910895CF92DF92EF9258
:101A9000FF920F931F93A89500EE17E021E430E02A
:101AA00048EC50E06AEA70E085E090E00E94A4040F
:101AB0000FEF1FEF21E430E048EC50E063E270E00C
:101AC00085E090E09DD920E530E040E550E065E01C
:101AD00070E08BEE90E094D9F0EECF2EF7E0DF2EA1
:101AE000A4E1EA2EF12C03E111E026E430E041E329
:101AF00051E066E470E085EF90E02EDAB7E1EB2E7E
:101B0000F12C24E430E04FE251E064E470E087EF30
:101B100090E022DA0FEF1FEF20E530E040E550E0E3
:101B200064E670E08BEE90E06BD915EAE12EF12CC3
:101B300003E111E023E730E041E351E063E770E0C7
:101B400085EF90E009DA83EAE82EF12C25E730E012
:101B50004FE251E065E770E087EF90E0FDD99EEC41
:101B6000E92E95E0F92E02E020EE37E040E050E06B
:101B700068EC70E08CE390E00E9499058091120679
:101B800090911306892B09F048C0E09171068E2FC1
:101B900090E08830910508F040C0FC01E25BFF4F07
:101BA0000C94F83EE3E9EE2EE4E0FE2E04C07EE85D
:101BB000E72E74E0F72E02E02FE130E04FEF5FEF09
:101BC00065E070E086E490E026C064E8E62E64E01C
:101BD000F62E18C05AE7E52E54E0F52E13C040E764
:101BE000E42E44E0F42E0EC036E6E32E34E0F32E6D
:101BF00009C02CE5E22E24E0F22E04C092E5E92E85
:101C000094E0F92E02E02FE130E04FEF5FEF65E066
:101C100070E08EE190E00E9499058091120690910B
:101C20001306019701F580911B06813069F038F0A9
:101C30008230C9F410E7E12E14E0F12E09C084E8E7
:101C4000E82E84E0F82E04C00AE7E02E04E0F02E2F
:101C500002E02FE130E04FEF5FEF65E070E08EE1F2
:101C600090E00E94990580911206909113060297C8
:101C700001F580912206813069F038F08230C9F494
:101C8000F0E7EF2EF4E0FF2E09C0B4E8EB2EB4E04D
:101C9000FB2E04C0AAE7EA2EA4E0FA2E02E02FE110
:101CA00030E04FEF5FEF65E070E08EE190E00E9482
:101CB00099058091120690911306049701F5809181
:101CC0007C06813069F038F08230C9F460E7E62E96
:101CD00064E0F62E09C0E4E8EE2EE4E0FE2E04C037
:101CE0007AE7E72E74E0F72E02E02FE130E04FEFC5
:101CF0005FEF65E070E08EE190E00E9499058091D1
:101D0000120690911306059701F5809170068130B7
:101D100069F038F08230C9F430E7E32E34E0F32E76
:101D200009C054E8E52E54E0F52E04C04AE7E42E3D
:101D300044E0F42E02E02FE130E04FEF5FEF65E08A
:101D400070E08EE190E00E949905809112069091DA
:101D50001306069701F580916D06813069F038F021
:101D60008230C9F480E7E82E84E0F82E09C024E828
:101D7000E22E24E0F22E04C09AE7E92E94E0F92E38
:101D800002E02FE130E04FEF5FEF65E070E08EE1C1
:101D900090E00E9499051F910F91FF90EF90DF90C6
:101DA000CF900895EF92FF920F931F9380910906B1
:101DB00090910A060A97A8F48091E00581110CC061
:101DC0000FE110E02CE330E044E650E06BE470E01B
:101DD0008EE690E00E94A40481E08093E0051092DA
:101DE00014068091090690910A060A978A35910592
:101DF000A8F48091140681110CC00FE110E02CE3CF
:101E000030E044E650E06BE470E08EE690E00E9443
:101E1000A40481E0809314061092E00580910906E5
:101E200090910A0684369105A0F0809114068130C5
:101E300061F40FE110E02CE330E044E650E06BE4A5
:101E400070E08EE690E00E94A404109214061092B6
:101E5000E0058091100690911106019779F4E090C9
:101E60000906F0900A0603E02FE130E04FEF5FEF44
:101E700064E670E082E890E00E94DF058091100641
:101E800090911106892B79F4E0900906F0900A06EA
:101E900003E02FE130E040E058EF64E670E082E8D4
:101EA00090E00E94DF051F910F91FF90EF90089541
:101EB000EF92FF920F931F9380913E0690913F0601
:101EC0000A97A8F480910806811111C00FE110E073
:101ED00027E330E048E550E06BE970E088E090E00F
:101EE0000E94A40481E08093080610926E068091FF
:101EF0003E0690913F0684369105D8F480910906FC
:101F000090910A060A97A8F080916E06811111C07F
:101F10000FE110E027E330E048E550E06BE970E0C6
:101F200088E090E00E94A40481E080936E06109205
:101F3000080680913E0690913F0684369105A0F0F8
:101F400080916E06813061F40FE110E027E330E00C
:101F500048E550E06BE970E088E090E00E94A4045E
:101F600010926E0610920806E0903E06F0903F0632
:101F700003E02FE130E04FEF5FEF64EB70E08FE0C4
:101F800090E00E94DF051F910F91FF90EF90089560
:101F9000EF92FF920F931F9380912B0690912C0646
:101FA0000A97A8F480910F0681110CC00FE110E090
:101FB00024E230E04AE550E064E670E088E090E03A
:101FC0000E94A40481E080930F061092260680915F
:101FD0002B0690912C060A978A359105A8F48091DA
:101FE000260681110CC00FE110E024E230E04AE542
:101FF00050E064E670E088E090E00E94A40481E094
:102000008093260610920F0680912B0690912C0645
:1020100084369105A1F480912606813061F40FE1A8
:1020200010E024E230E04AE550E064E670E088E049
:1020300090E00E94A40410920F0610922606E090F1
:102040002B06F0902C0603E02FE130E04FEF5FEF1E
:102050006EE670E084E190E00E94DF0580917D06ED
:1020600090917E060A97A8F480917706811111C09D
:102070000FE110E024E230E04AE550E064E670E071
:102080008FED90E00E94A40481E080937706109287
:10209000400680917D0690917E060A978A359105CB
:1020A000A8F480914006811111C00FE110E024E2F4
:1020B00030E04AE550E064E670E08FED90E00E9489
:1020C000A40481E08093400610927706E0907D069C
:1020D000F0907E0684E6E816F10421F4109277066B
:1020E0001092400603E02FE130E04FEF5FEF6EE625
:1020F00070E089EE90E00E94DF051F910F91FF9044
:10210000EF900895CF93DF9300D000D0CDB7DEB726
:10211000809163001C821B821A821982BE016F5F4C
:102120007F4FCE0103960E945B3D8B819C81883757
:102130009540A0F4A89589819A81843C994070F4D7
:10214000A89589819A818D3D954040F0A89581E0C0
:1021500090E09093110680931006A8950F900F9031
:102160000F900F90DF91CF910895CF93DF9300D020
:1021700000D0CDB7DEB7A895809163001C821B828A
:102180001A821982BE016F5F7F4FCE0103960E94B3
:102190005B3D8B819C818837954070F489819A8161
:1021A000843C994048F489819A818D3D954020F086
:1021B00010921106109210060F900F900F900F9032
:1021C000DF91CF9108957F928F929F92AF92BF92AD
:1021D000CF92DF92EF92FF920F931F93CF93DF93F3
:1021E000EC016B015A014901702EA8958091E3051D
:1021F0009091E4050A97A8F480917206811111C0AC
:102200000FE110E02EE130E044E650E06550710946
:10221000CE0144970E94A40481E08093720610923C
:1022200033068091E3059091E4050A978A3591057C
:10223000C0F480913306811114C00FE110E02EE14B
:1022400030E044E650E0B60165507109CE01449794
:102250000E94A40481E080933306109272061092CB
:102260000B068091E3059091E40584369105C0F05A
:1022700080910B06811114C00FE110E02EE130E0D7
:1022800044E650E0B60165507109CE0144970E94C2
:10229000A40481E080930B0610923306109272061C
:1022A000E090E305F090E405072D9401A501B60147
:1022B000CE010E94DF05A895DF91CF911F910F916C
:1022C000FF90EF90DF90CF90BF90AF909F908F9056
:1022D0007F900895A89580913006813071F4A49A7A
:1022E00080E185BBA8952FEF82E597E021508040E3
:1022F0009040E1F700C0000015BAA8950895A89590
:1023000080913006813021F5A49A80E185BB2FEFC2
:1023100032E597E0215030409040E1F700C00000E6
:10232000A89515BA2FEF32E597E021503040904044
:10233000E1F700C00000A89585BB2FEF32E587E0EC
:10234000215030408040E1F700C00000A89515BA48
:102350000895A89580913006813009F048C0A49A6C
:1023600080E185BBA8952FEF32E597E02150304002
:102370009040E1F700C00000A89515BAA8952FEF8E
:1023800032E597E0215030409040E1F700C0000076
:10239000A89585BBA8952FEF32E597E021503040F6
:1023A0009040E1F700C00000A89515BAA8952FEF5E
:1023B00032E597E0215030409040E1F700C0000046
:1023C000A89585BB2FEF32E587E021503040804053
:1023D000E1F700C00000A89515BA9FEF22E537E0AD
:1023E000915020403040E1F700C00000A8950895CA
:1023F000A89510922D0610921F061092DE051092DD
:10240000430610921C0610920E0610922F06109290
:10241000250610923D061092DF0583EB92E00E94A4
:10242000134280933006A89584EB92E00E941B42F1
:102430009093210680932006A89580911206909192
:102440001306892B51F5A895E09171068E2F90E027
:102450008830910510F5FC01EA5AFF4F4EE150E03B
:102460000C94F83E64E972E014C066E772E011C0B3
:1024700068E572E00EC06AE372E00BC06CE172E0E6
:1024800008C06EEF71E005C060EE71E002C062EC62
:1024900071E089EE95E00E940342A89580911206B2
:1024A000909113060197D1F4A89580911B06813075
:1024B00069F038F0823091F44EE150E068E671E066
:1024C00009C04EE150E064EA71E004C04EE150E022
:1024D00066E871E089EE95E00E940342A89580913C
:1024E0001206909113060297D1F4A89580912206C6
:1024F000813069F038F0823091F44EE150E06EE0C6
:1025000071E009C04EE150E06AE471E004C04EE1C0
:1025100050E06CE271E089EE95E00E940342A895DC
:1025200080911206909113060497C9F480917C065D
:10253000813069F038F0823091F44EE150E064EB84
:1025400070E009C04EE150E060EF70E004C04EE181
:1025500050E062ED70E089EE95E00E940342A8959C
:1025600080911206909113060597C9F48091700628
:10257000813069F038F0823091F44EE150E06AE544
:1025800070E009C04EE150E066E970E004C04EE141
:1025900050E068E770E089EE95E00E940342A8955C
:1025A00080911206909113060697C9F480916D06EA
:1025B000813069F038F0823091F44EE150E060E013
:1025C00070E009C04EE150E06CE370E004C04EE101
:1025D00050E06EE170E089EE95E00E940342A8951C
:1025E00087EC90E00197F1F700C000008091E905C9
:1025F0009091EA059093DD058093DC058091EB05D1
:102600009091EC0590933206809331068091ED0510
:102610009091EE0590937A06809379068091EF056C
:102620009091F00590931A06809319068091F10518
:10263000809346068091F3059091F40590931806D7
:10264000809317068091F5059091F60590932A06E0
:10265000809329068091F7059091F80590932806BC
:10266000809327068091F9058093D8058091FB051A
:102670009091FC0590936A06809369068091FD0510
:102680009091FE0590934506809344068091120632
:1026900090911306079741F48091FF0590910006F1
:1026A0009093130680931206809101069091020682
:1026B00090936806809367068091030690910406C4
:1026C0009093E8058093E7058091050690910606B2
:1026D00090930D0680930C06A895089510927E069F
:1026E00010927D06BC9A80917D06880F81BF109262
:1026F0002C0610922B06139A80912B06880F80933C
:10270000860027DE8DE490E0909374068093730634
:1027100081E090E090931106809310060895CF9386
:10272000BC9A80917D06880F81BF139A80912B06F9
:10273000880F809386008091120690911306892B52
:1027400009F0F3C14091E3055091E4052091190689
:1027500030911A06429FC001439F900D529F900DE9
:1027600011246AE070E00E94E43E70934206609398
:10277000410680912B0690912C068536910530F00C
:1027800084E690E090932C0680932B0620912706F8
:102790003091280680912B0690912C062817390736
:1027A00020F430932C0620932B0680912D06811166
:1027B00013C080913E0690913F068233910538F414
:1027C00084E690E090932C0680932B0605C0C29778
:1027D00019F081E080932D0680912D06E09131065D
:1027E000F0913206813051F56E177F0738F5409130
:1027F0003E0650913F0680912B0690912C0646177D
:102800005707B8F401962817390728F090932C063B
:1028100080932B0604C030932C0620932B068091C6
:102820002B0690912C068536910540F084E690E0C9
:1028300001C0019790932C0680932B06E617F707AB
:1028400098F540913E0650913F064E175F07C8F439
:1028500080912B0690912C0601968536910510F0FB
:1028600084E690E090932C0680932B0680912B06B3
:1028700090912C062817390720F430932C062093CA
:102880002B06E417F50780F480912B0690912C0617
:102890004E1B5F0B4B30510510F4019701C00B9795
:1028A00090932C0680932B06C0914606C130D1F43C
:1028B00080911F06811116C02091090630910A06E9
:1028C00080911706909118062817390759F48091BE
:1028D0003E0690913F069093320680933106FADCD3
:1028E000C0931F06C091D805C13009F58091DE055F
:1028F00081111DC08091090690910A0620916906F8
:1029000030916A06821B930B059788F4209131065B
:10291000309132068091440690914506820F931FB4
:102920009093320680933106D5DCC093DE0580910A
:10293000430681111CC08091090690910A062091DE
:10294000170630911806821B930B029780F482E3DE
:1029500090E090937E0680937D0681E0809343060D
:1029600080930E0680914606811101C0B3DC209150
:1029700017063091180660917506709176064091A1
:10298000790650917A06649FC001659F900D749FEF
:10299000900D11246AE070E00E94E43E620F731F04
:1029A0007093DB056093DA05E0917D06F0917E0679
:1029B0004091DC055091DD054617570720F45093F0
:1029C000DB054093DA058091290690912A068E173F
:1029D0009F0720F490937E0680937D0680910906E0
:1029E00090910A062817390700F520913D0621111C
:1029F0001CC084179507C8F46091DA057091DB0557
:102A000020917D0630917E068617970740F42F5F50
:102A10003F4F2536310528F024E630E002C0215032
:102A2000310930937E0620937D064817590768F5D3
:102A300020917D0630917E06841B950B069718F435
:102A40002150310902C02B50310930937E0620936A
:102A50007D068091DF05811106C051DC81E0809305
:102A600025068093DF052091E5053091E6058091EC
:102A70002006909121068217930738F42FDE81E01B
:102A800090E0909311068093100680911C068111AE
:102A90004CC040916706509168068091170690914E
:102AA00018068417950708F040C0E0910906F091D8
:102AB0000A064E175F0729F481E080933D06809354
:102AC0002F0680913D06813081F56091E10570917E
:102AD000E2052091E7053091E8056217730798F445
:102AE00080917D0690917E06E417F50738F40196F3
:102AF0008536910520F084E690E001C0019790931F
:102B00007E0680937D062617370778F410923D06DF
:102B10008091750690917606821B930B90937606B2
:102B20008093750681E080931C0680911206909137
:102B30001306019709F001C110922C0610922B0682
:102B40008091430681111BC02091090630910A062D
:102B500080911706909118068217930780F482E3FC
:102B600090E090937E0680937D0681E080934306FB
:102B700080930E0680914606811101C0ABDB209147
:102B8000170630911806609175067091760640918F
:102B9000790650917A06649FC001659F900D749FDD
:102BA000900D11246AE070E00E94E43E620F731FF2
:102BB0007093DB056093DA05E0917D06F0917E0667
:102BC0004091DC055091DD054617570720F45093DE
:102BD000DB054093DA058091290690912A068E172D
:102BE0009F0720F490937E0680937D0680910906CE
:102BF00090910A062817390700F520913D0621110A
:102C00001CC084179507C8F46091DA057091DB0544
:102C100020917D0630917E068617970740F42F5F3E
:102C20003F4F2536310528F024E630E002C0215020
:102C3000310930937E0620937D064817590768F5C1
:102C400020917D0630917E06841B950B069718F423
:102C50002150310902C02B50310930937E06209358
:102C60007D068091DF05811106C049DB81E08093FC
:102C700025068093DF052091E5053091E6058091DA
:102C80002006909121068217930738F427DD81E012
:102C900090E0909311068093100680911C0681119C
:102CA0004CC040916706509168068091170690913C
:102CB00018068417950708F040C0E0910906F091C6
:102CC0000A064E175F0729F481E080933D06809342
:102CD0002F0680913D06813081F56091E10570916C
:102CE000E2052091E7053091E8056217730798F433
:102CF00080917D0690917E06E417F50738F40196E1
:102D00008536910520F084E690E001C0019790930C
:102D10007E0680937D062617370778F410923D06CD
:102D20008091750690917606821B930B90937606A0
:102D30008093750681E080931C0680911206909125
:102D40001306029709F00FC110927E0610927D06BD
:102D5000C0914606C130D1F480911F06811116C082
:102D60002091090630910A06809117069091180665
:102D70002817390759F480913E0690913F069093A9
:102D8000320680933106A6DAC0931F064091E30510
:102D90005091E4052091190630911A06429FC00116
:102DA000439F900D529F900D11246AE070E00E94A5
:102DB000E43E709342066093410680912B06909109
:102DC0002C068536910530F084E690E090932C0631
:102DD00080932B06809127069091280620912B0640
:102DE00030912C068217930720F490932C06809341
:102DF0002B0620912D06211114C020913E06309102
:102E00003F062639310538F424E630E030932C06AD
:102E100020932B0606C02639310519F021E02093B6
:102E20002D0620912D064091310650913206213019
:102E300061F56417750748F5E0913E06F0913F068D
:102E400020912B0630912C06E617F707C0F42F5F70
:102E50003F4F8217930728F030932C0620932B06C0
:102E600004C090932C0680932B0620912B06309162
:102E70002C062536310548F024E630E002C021500A
:102E8000310930932C0620932B064617570708F07C
:102E90006AC02091460621112CC020913E06309137
:102EA0003F0624173507D0F460912B0670912C064D
:102EB0006F5F7F4F6536710510F064E670E07093C8
:102EC0002C0660932B0660912B0670912C068617BA
:102ED000970720F490932C0680932B0642175307F4
:102EE00008F041C080912B0690912C06241B350BD5
:102EF00030C02130C1F52091090630910A06609159
:102F000017067091180626173707D0F440912B0644
:102F100050912C064F5F5F4F4536510510F044E647
:102F200050E050932C0640932B0640912B06509175
:102F30002C068417950720F490932C0680932B067B
:102F40006217730780F480912B0690912C06261B44
:102F5000370B2B30310510F4019701C00B9790937C
:102F60002C0680932B0680911206909113068430D4
:102F7000910521F08530910509F0DAC04091E30513
:102F80005091E4052091190630911A06429FC00124
:102F9000439F900D529F900D11246AE070E00E94B3
:102FA000E43E709342066093410680912B06909117
:102FB0002C068536910530F084E690E090932C063F
:102FC00080932B06E0912706F091280680912B062E
:102FD00090912C06E817F90720F4F0932C06E09363
:102FE0002B0620912D0680913E0690913F062111DF
:102FF00010C08639910538F424E630E030932C0671
:1030000020932B0606C08639910519F021E0209304
:103010002D0620912D064091310650913206213027
:1030200041F56417750728F520912B0630912C0681
:1030300086179707C0F42F5F3F4FE217F30728F07A
:1030400030932C0620932B0604C0F0932C06E093BB
:103050002B0620912B0630912C062536310548F0A1
:1030600024E630E002C02150310930932C06209331
:103070002B064617570738F12091290630912A066A
:1030800060917D0670917E062617370720F43093F5
:103090007E0620937D064817590708F0FFC08091EF
:1030A0007D0690917E06019690937E0680937D0624
:1030B0008536910508F4F2C084E690E090937E0690
:1030C00080937D06EBC084179507D0F420912B06E2
:1030D00030912C062F5F3F4F2536310510F024E646
:1030E00030E030932C0620932B0620912B06309154
:1030F0002C06E217F30720F4F0932C06E0932B063E
:103100004817590708F0B8CF20912B0630912C06AC
:10311000BC01641B750B6B30710538F02B50310905
:1031200030932C0620932B06A7CF21503109F8CFDE
:10313000069709F0B3C04091E3055091E405209152
:10314000190630911A06429FC001439F900D529F6D
:10315000900D11246AE070E00E94E43E70934206F4
:103160006093410680912B0690912C06853691053F
:1031700030F084E690E090932C0680932B0620910B
:1031800027063091280680912B0690912C0628174F
:10319000390720F430932C0620932B0680912D06BE
:1031A000811114C080913E0690913F0686399105A9
:1031B00038F484E690E090932C0680932B0606C0AA
:1031C0008639910519F081E080932D0680912D06B6
:1031D000E0913106F0913206813051F56E177F078C
:1031E00038F540913E0650913F0680912B06909114
:1031F0002C0646175707B8F401962817390728F008
:1032000090932C0680932B0604C030932C062093B9
:103210002B0680912B0690912C068536910540F067
:1032200084E690E001C0019790932C0680932B06D2
:10323000E617F70798F540913E0650913F064E1766
:103240005F07C8F480912B0690912C060196853675
:10325000910510F084E690E090932C0680932B0665
:1032600080912B0690912C062817390720F4309373
:103270002C0620932B06E417F50780F480912B068B
:1032800090912C064E1B5F0B4B30510510F40197AB
:1032900001C00B9790932C0680932B06CF91089535
:1032A00063EC70E084E992E00E94364262EC71E0E7
:1032B00086E992E00E94364266E170E088E992E099
:1032C0000E94364266E170E08AE992E00E9436424E
:1032D00061E070E08CE992E00E943642A8956EE6CB
:1032E00070E08EE992E00E94364264E670E080EA87
:1032F00092E00E94364264E670E082EA92E00E9428
:10330000364260E070E084EA92E00E943642A8957E
:1033100060E070E086EA92E00E94364260E070E091
:1033200088EA92E00E94364260E070E08AEA92E029
:103330000E94364260E070E08CEA92E00E943642E1
:1033400060E070E08EEA92E00E94364260E070E059
:1033500080EB92E00E943642A89566EE70E086E728
:1033600092E00E94364262EC71E088E792E00E94AF
:10337000364266E170E08AE792E00E94364266E1FA
:1033800070E08CE792E00E94364261E070E08EE7E8
:1033900092E00E943642A89563E770E080E892E0F0
:1033A0000E94364264E670E082E892E00E94364273
:1033B00064E670E084E892E00E94364260E070E0EB
:1033C00086E892E00E94364260E070E088E892E091
:1033D0000E94364260E070E08AE892E00E94364245
:1033E000A89560E070E08CE892E00E94364260E0D0
:1033F00070E08EE892E00E94364260E070E080E982
:1034000092E00E94364260E070E082E992E00E9421
:103410003642A89566EE70E088E592E00E9436425A
:1034200062EC71E08AE592E00E94364266E170E06B
:103430008CE592E00E94364266E170E08EE592E013
:103440000E94364261E070E080E692E00E943642DF
:10345000A89563E770E082E692E00E94364264E657
:1034600070E084E692E00E94364264E670E086E610
:1034700092E00E94364260E070E088E692E00E94AE
:10348000364260E070E08AE692E00E94364260E0F8
:1034900070E08CE692E00E943642A89560E070E011
:1034A0008EE692E00E94364260E070E080E792E0B3
:1034B0000E94364260E070E082E792E00E9436426D
:1034C00060E070E084E792E00E943642A89566E9E9
:1034D00070E08AE392E00E94364268EC70E08CE390
:1034E00092E00E94364266E170E08EE392E00E9434
:1034F000364266E170E080E492E00E94364261E08C
:1035000070E082E492E00E943642A89563E770E0A2
:1035100084E492E00E94364264E670E086E492E041
:103520000E94364264E670E088E492E00E943642EF
:1035300060E070E08AE492E00E94364260E070E071
:103540008CE492E00E94364260E070E08EE492E00B
:103550000E943642A89560E070E080E592E00E940B
:10356000364260E070E082E592E00E94364260E020
:1035700070E084E592E00E94364260E070E086E50B
:1035800092E00E943642A8956EEB70E08CE192E0EA
:103590000E94364268EC70E08EE192E00E94364272
:1035A00066E170E080E292E00E94364266E170E0FF
:1035B00082E292E00E94364261E070E084E292E0B2
:1035C0000E943642A89564E670E086E292E00E948E
:1035D000364264E670E088E292E00E94364264E699
:1035E00070E08AE292E00E94364260E070E08CE295
:1035F00092E00E94364260E070E08EE292E00E942B
:10360000364260E070E080E392E00E943642A89586
:1036100060E070E082E392E00E94364260E070E099
:1036200084E392E00E94364260E070E086E392E03C
:103630000E94364260E070E088E392E00E943642E9
:10364000A89566EE70E08EEF91E00E94364262EC43
:1036500071E080E092E00E94364266E170E082E034
:1036600092E00E94364266E170E084E092E00E94BF
:10367000364261E070E086E092E00E943642A89512
:1036800063E770E088E092E00E94364264E670E012
:103690008AE092E00E94364264E670E08CE092E0BC
:1036A0000E94364260E070E08EE092E00E94364276
:1036B00060E070E080E192E00E94364260E070E0FD
:1036C00082E192E00E943642A89560E070E084E1D9
:1036D00092E00E94364260E070E086E192E00E9453
:1036E000364260E070E088E192E00E94364260E09D
:1036F00070E08AE192E00E943642A89566EE70E0A2
:1037000080EE91E00E94364262EC71E082EE91E040
:103710000E94364266E170E084EE91E00E943642FB
:1037200066E170E086EE91E00E94364261E070E072
:1037300088EE91E00E943642A89563E770E08AEE39
:1037400091E00E94364264E670E08CEE91E00E94C7
:10375000364264E670E08EEE91E00E94364260E010
:1037600070E080EF91E00E94364260E070E082EF0E
:1037700091E00E94364260E070E084EF91E00E94A8
:103780003642A89560E070E086EF91E00E943642F4
:1037900060E070E088EF91E00E94364260E070E007
:1037A0008AEF91E00E94364260E070E08CEF91E099
:1037B0000E943642A89563EC70E084EA91E00E9492
:1037C000364266E170E088EA91E00E94364261E0AC
:1037D00070E08CEA91E00E9436426FE070E08EEA81
:1037E00091E00E943642A89564E670E080EB91E09B
:1037F0000E94364261E070E08AEB91E00E9436421E
:1038000063EC70E08CEB91E00E9436426AE070E07D
:103810008EEB91E00E943642A89562EC71E08CE458
:1038200091E00E94364266E170E080E591E00E94FE
:10383000364261E070E082E591E00E9436426EE639
:1038400070E084E591E00E943642A89564E670E05D
:1038500088E591E00E94364262E070E080E691E007
:103860000E94364262EC71E082EF90E00E943642A4
:1038700066E170E084EF90E00E94364262E170E021
:1038800086EF90E00E943642A89564E670E08CEFE7
:1038900090E00E94364264E670E08EEF90E00E9475
:1038A000364264E070E086E091E00E9436426CE2CD
:1038B00071E08CE091E00E943642A89562EC71E0E4
:1038C00088E990E00E94364266E170E08AE990E083
:1038D0000E94364266E170E08CE990E00E94364238
:1038E00061E070E08EE990E00E943642A8956EE6B5
:1038F00070E080EA90E00E94364264E670E082EA7E
:1039000090E00E94364264E670E084EA90E00E9413
:10391000364265E070E08CEA90E00E943642A8955D
:1039200062EC71E08EE390E00E94364266E170E066
:1039300082E490E00E94364261E070E084E490E02E
:103940000E9436426EE670E086E490E00E943642C5
:10395000A89564E670E08AE490E00E94364266E052
:1039600070E082E590E00E94364263EC70E084E90A
:1039700092E00E943642A89508956FE070E088EBCF
:1039800092E00E9436426FE070E086EB92E00E9487
:1039900036426FE070E084EB92E00E94364261E0D4
:1039A00083EB92E00E94294261E082EB92E00C946A
:1039B00029428FB9779BFECF8FB10895CF93A39AF9
:1039C000AB9AAB9880E0F5DFC82F80E0F2DFAB9ACE
:1039D0006C2F70E0762F6627682B687F7F7723E057
:1039E000769567952A95E1F780E090E00E94F33D97
:1039F00020E030E040E85EE30E94593E0E94C73D6F
:103A000070930A0660930906CB01CF910895CF9376
:103A1000A79AAF9AAF9880E0CCDFC82F80E0C9DFCB
:103A2000AF9A6C2F70E0762F6627682B687F7F77C0
:103A300023E0769567952A95E1F780E090E00E9473
:103A4000F33D20E030E040E85EE30E94593E0E94F2
:103A5000C73D70933F0660933E06CB01CF9108951A
:103A600080E091E0909383068093820680910A061D
:103A70008F93809109068F938EE091E09F938F93AF
:103A80000E94333F8DE08A95F1F700008091E405B4
:103A90008F938091E3058F9388E191E09F938F93BB
:103AA0000E94333F9DE09A95F1F7000080912C062B
:103AB0008F9380912B068F9382E291E09F938F9357
:103AC0000E94333F8DE08A95F1F7000080917E06D9
:103AD0008F9380917D068F938DE291E09F938F93DA
:103AE0000E94333F9DE09A95F1F7000087E391E053
:103AF0009F938F930E94333F8DE08A95F1F70000EA
:103B000080913F068F9380913E068F938FE391E0E3
:103B10009F938F930E94333F8DB79EB746960FB603
:103B2000F8949EBF0FBE8DBF809110069091110634
:103B3000892B41F488E491E09F938F930E94333F57
:103B40000F900F908091100690911106019741F40B
:103B50008FE491E09F938F930E94333F0F900F90DB
:103B60009DE09A95F1F70000E0911206F09113069E
:103B7000E830F10508F08FC0E25AFF4F0C94F83E90
:103B800086E591E09F938F930E94333F0F900F90B3
:103B9000E09171068E2F90E08830910508F07BC08F
:103BA000FC01EA59FF4F0C94F83E85E691E06DC0A8
:103BB00085E791E06AC08DEA91E067C08CEB91E007
:103BC00064C08BEC91E061C08AED91E09F938F938C
:103BD0000E94333F0F900F9080911B06813009F4B3
:103BE0004CC008F447C0823009F44AC008958AEEF8
:103BF00091E09F938F930E94333F0F900F9080919D
:103C000022068130D1F1B0F18230D1F108958BEFED
:103C100091E03BC089E092E09F938F930E94333FF5
:103C20000F900F9080917C06813039F118F182302D
:103C300039F108958AE192E09F938F930E94333F78
:103C40000F900F90809170068130B9F098F082301B
:103C5000B9F008958DE292E09F938F930E94333FD5
:103C60000F900F9080916D06813039F018F08230FE
:103C700039F0089580E891E008C08FE891E005C030
:103C80008EE991E002C08FE392E09F938F930E94B0
:103C9000333F0F900F900895CF92DF92EF92FF92F3
:103CA0000F931F93CF93DF9300D000D0CDB7DEB733
:103CB0008091100690911106019709F00EC1809134
:103CC000230690912406892BC9F40FE110E024E229
:103CD00030E04AE550E064E670E088E090E00E9461
:103CE000A40424E230E04AE550E064E670E08FEDA1
:103CF00090E00E94A404A8950E94EB07CC24C394F2
:103D0000D12C8091100690911106019709F0E5C021
:103D1000A895A6DE80917306909174068A35910568
:103D200049F42FEF8DE399E4215080409040E1F772
:103D300000C00000A89503E02FE130E04FEF5FEFF7
:103D400069E170E085E890E00E94E31080916300F3
:103D5000A8951C821B821A821982BE016F5F7F4F59
:103D6000CE0103960E945B3D8B819C81853C9940EE
:103D700088F089819A81883D9E4060F489819A818A
:103D8000853C994038F0D0922406C09223061092C8
:103D90003506F1D38B819C81853C994008F43FC066
:103DA00089819A818C3D9540D0F589819A81853FA2
:103DB0009140A8F1D0922406C092230610924706A3
:103DC0008091120690911306892B11F40E94AA2F5C
:103DD0008091120690911306019711F40E946A389F
:103DE0008091120690911306029711F40E94713986
:103DF0008091120690911306049711F40E94763A6E
:103E00008091120690911306059709F43CD5809194
:103E1000120690911306069711F40E94A22ECEDD91
:103E20000E94D20EA8958FEF91EE24E08150904031
:103E30002040E1F700C00000EADDA8950E94580F7D
:103E4000E0902B06F0902C0603E02FE130E04FEFDE
:103E50005FEF6EE670E08CE190E00E94DF05E0909D
:103E60007D06F0907E062FE130E04FEF5FEF6EE6CB
:103E700070E080EF90E00E94DF050E94B510809115
:103E8000100690911106892B09F03BCF0E946A1110
:103E9000A8950E94F811A8950E94EB070FE110E089
:103EA00024E230E04AE550E064E670E088E090E02B
:103EB0000E94A40424E230E04AE550E064E670E0A9
:103EC0008FED90E00E94A4041092E4051092E305A7
:103ED000109224061092230614CF0F900F900F908B
:103EE0000F90DF91CF911F910F91FF90EF90DF9096
:103EF000CF900895EF92FF920F931F93CF938091ED
:103F00003406813009F04BC18FE190E00E94190620
:103F10000E94C10B85E080933A06C5E0809134068B
:103F2000813009F03CC10E94DD0C80913A0682305C
:103F3000D9F4809166068F5F809366060FE110E0EA
:103F40002CE330E046EE50E069E670E081E090E07E
:103F50000E94A40422E330E043EC50E068E270E009
:103F600088E090E00E94A40480913A068330D9F45E
:103F7000809166068150809366060FE110E02CE385
:103F800030E046EE50E069E670E081E090E00E94AB
:103F9000A40422E330E043EC50E068E270E088E003
:103FA00090E00E94A40480916606853010F0109283
:103FB000660680916606823081F1B8F48823D9F0D4
:103FC000813009F0C1C075E8E72E75E0F72E01E0F9
:103FD0002FE130E04FEF5FEF6CE370E088E090E0BE
:103FE0000E94990586EB92E029C08330B1F18430BC
:103FF00009F471C0A9C0EEE9EE2EE5E0FE2E01E065
:104000002FE130E04FEF5FEF6CE370E08FE090E086
:104010000E94990588EB92E011C069E7E62E65E001
:10402000F62E01E02FE130E04FEF5FEF6CE370E040
:1040300082E390E00E94990584EB92E00E941B428B
:104040007C0103E02FE130E04FEF5FEF62E870E0CA
:1040500080E590E00E94DF0577C041E6E42E45E070
:10406000F42E01E02FE130E04FEF5FEF6CE370E002
:1040700088E290E00E9499055FE6E52E55E0F52E76
:1040800002E02FE130E04FEF5FEF62E870E088E29E
:1040900090E00E94990580913A06811119C000D9DB
:1040A0006CDC3BE2E32E35E0F32E2FE130E04FEF06
:1040B0005FEF62E870E088E290E00E9499052FEFE0
:1040C00089E698E1215080409040E1F700C000006F
:1040D000C0933A0639C020E5E22E25E0F22E01E039
:1040E0002FE130E04FEF5FEF6CE370E08EE190E0A6
:1040F0000E94990583EB92E00E941342813079F48B
:1041000092E4E92E95E0F92E03E02FE130E04FEF45
:104110005FEF62E870E080E590E00E94990583EB34
:1041200092E00E94134281110FC08DE3E82E85E0DA
:10413000F82E03E02FE130E04FEF5FEF62E870E030
:1041400080E590E00E94990580913A06813089F4DB
:104150001092340610922406109223068FE190E00C
:104160000E94190681E090E090931106809310065A
:1041700093DD80913A06811106C081E08093340678
:104180001092780612D0C0933A062FE785EB91E0A3
:10419000215080409040E1F700C00000BFCECF9199
:1041A0001F910F91FF90EF900895BF92CF92DF92F1
:1041B000EF92FF920F931F93CF93DF938091780636
:1041C0008111CFC185E080933A06C9E1D0E025E0B6
:1041D000C22ED12C35E0B32E809178068111C1C159
:1041E00080916606813009F46FC038F0823009F49E
:1041F000DDC0843009F441C1A4C188EB92E00E9483
:104200001B427C0103E02FE130E040E058EF62E820
:1042100070E080E590E00E94DF0588EB92E00E946C
:104220001B4290933906809338060E94DD0C8091E2
:104230003A068230A9F480913806909139060196A9
:1042400090933906809338060FE110E02CE330E0BC
:1042500046EE50E069E670E081E090E00E94A40440
:1042600080913A068330A9F48091380690913906FE
:10427000019790933906809338060FE110E02CE304
:1042800030E046EE50E069E670E081E090E00E94A8
:10429000A40480913806909139064A9720F0D09373
:1042A0003906C093380680913806909139060A97EE
:1042B00020F4D0933906C093380660913806709187
:1042C000390688EB92E066C086EB92E00E941B42C2
:1042D0007C0103E02FE130E040E058EF62E870E05D
:1042E00080E590E00E94DF0586EB92E00E941B4291
:1042F00090931606809315060E94DD0C80913A0675
:104300008230A9F48091150690911606019690933B
:104310001606809315060FE110E02CE330E046EE20
:1043200050E069E670E081E090E00E94A404809192
:104330003A068330A9F480911506909116060197EC
:1043400090931606809315060FE110E02CE330E001
:1043500046EE50E069E670E081E090E00E94A4043F
:1043600080911506909116064A9720F0D093160674
:10437000C093150680911506909116060A9720F4B1
:10438000D0931606C0931506609115067091160617
:1043900086EB92E00E9436422FE788E391E02150BD
:1043A00080409040E1F700C00000CBC084EB92E079
:1043B0000E941B427C0103E02FE130E040E058EF17
:1043C00062E870E080E590E00E94DF0584EB92E017
:1043D0000E941B4290933706809336060E94DD0CA4
:1043E00080913A068230A9F4809136069091370682
:1043F000019690933706809336060FE110E02CE388
:1044000030E046EE50E069E670E081E090E00E9426
:10441000A40480913A068330A9F4809136069091E5
:104420003706019790933706809336060FE110E028
:104430002CE330E046EE50E069E670E081E090E089
:104440000E94A40480913606909137064F9720F081
:10445000D0923706C0923606809136069091370684
:10446000059720F4D0923706C09236066091360642
:104470007091370684EB92E08DCF83EB92E00E943F
:1044800013428093D9050E94DD0C80913A06823058
:1044900089F48091D9058F5F8093D9050FE110E0F1
:1044A0002CE330E046EE50E069E670E081E090E019
:1044B0000E94A40480913A06833089F48091D90542
:1044C00081508093D9050FE110E02CE330E046EEF7
:1044D00050E069E670E081E090E00E94A4048091E1
:1044E000D905823010F01092D9058091D90581301C
:1044F00079F492E4E92E95E0F92E03E02FE130E023
:1045000040E058EF62E870E080E590E00E94990595
:104510008091D90581110FC08DE3E82E85E0F82E3A
:1045200003E02FE130E040E058EF62E870E080E522
:1045300090E00E9499056091D90583EB92E00E947A
:10454000294280913A06813049F48093780680931D
:1045500034068FE190E00E941906CCDCB0923A0656
:104560003BCEDF91CF911F910F91FF90EF90DF90A5
:10457000CF90BF9008954F925F926F927F928F92EB
:104580009F92AF92BF92CF92DF92EF92FF920F93E2
:104590001F93CF93DF9380913506811163C18FE123
:1045A00090E00E9419060E94330B85E080933A0642
:1045B0001092340610922E0655245394C7E0D0E092
:1045C000A6E0CA2ED12CB5E0AB2EB12C14E0812E82
:1045D000912C03E0602E712C85E0482E80913506E9
:1045E000811140C10E94DD0C80913A06823089F42D
:1045F00080912E068F5F80932E060FE110E02CE352
:1046000030E046EE50E069E670E081E090E00E9424
:10461000A40480913A06833089F480912E0681505B
:1046200080932E060FE110E02CE330E046EE50E0E0
:1046300069E670E081E090E00E94A40480912E067B
:10464000893010F010922E06E0912E068E2F90E009
:104650008930910508F0D4C0FC01E259FF4F0C9459
:10466000F83EFDE0EF2EF5E0FF2E02E02FE130E016
:104670004FEF5FEF62E870E088E090E00E949905FC
:10468000109234061092130610921206B9C0EFEF82
:10469000EE2EE4E0FE2E02E02FE130E04FEF5FEF80
:1046A00068E770E088E090E00E9499051092340677
:1046B00081E090E013C071EFE72E74E0F72E02E086
:1046C0002FE130E04FEF5FEF68E770E088E090E0C7
:1046D0000E9499051092340682E090E090931306B0
:1046E000809312068DC065EEE62E64E0F62E02E0A1
:1046F0002FE130E04FEF5FEF68E770E088E090E097
:104700000E94990510923406709213066092120668
:1047100077C053EDE52E54E0F52E02E02FE130E0B6
:104720004FEF5FEF68E770E088E090E00E94990546
:1047300010923406909213068092120661C03DECEE
:10474000E32E34E0F32E02E02FE130E04FEF5FEF95
:104750006EE670E088E290E00E94990543ECE42E5A
:1047600044E0F42E2FE130E04FEF5FEF67E870E0B8
:104770008FE090E00E94990510923406B0921306E3
:10478000A09212063DC026EBE22E24E0F22E02E0BB
:104790002FE130E04FEF5FEF68E770E088E090E0F6
:1047A0000E94990510923406D0921306C092120608
:1047B00027C098E9E92E94E0F92E02E02FE130E0DD
:1047C0004FEF5FEF68E770E088E090E00E949905A6
:1047D00010923406D0931306C093120611C082EAD9
:1047E000E82E84E0F82E02E02FE130E04FEF5FEF9B
:1047F00068E770E082E090E00E94990550923406EC
:1048000080913A06813011F580913406813059F457
:104810001092130610921206109235068FE190E066
:104820000E94190667DB50923506109224061092FA
:1048300023068091120690911306909300068093B0
:10484000FF058FE190E00E94190626DA40923A06B1
:104850002FEF80E792E0215080409040E1F700C0C8
:104860000000BCCEDF91CF911F910F91FF90EF9090
:10487000DF90CF90BF90AF909F908F907F906F9080
:104880005F904F900895EF92FF920F931F93CF93F5
:10489000DF93A895809147068111F4C08FE190E0E5
:1048A0000E9419060E944F0C8091700690E0909330
:1048B0001E0680931D0685E080933A06C1E0D5E090
:1048C000809147068111DEC0A8950E94DD0C809181
:1048D0003A068230A9F480911D0690911E06019639
:1048E00090931E0680931D060FE110E02CE330E04C
:1048F00046EE50E069E670E081E090E00E94A4049A
:1049000080913A068330A9F480911D0690911E068D
:10491000019790931E0680931D060FE110E02CE393
:1049200030E046EE50E069E670E081E090E00E9401
:10493000A40480911D0690911E06039720F010920A
:104940001E0610921D0680911D0690911E06813054
:10495000910589F1D0F0029709F046C080E7E82E72
:1049600084E0F82E02E02FE130E04FEF5FEF6DE7DB
:1049700070E088E290E00E94990582E080937006E2
:104980004EE150E06AE570E02BC024E8E22E24E01E
:10499000F22E02E02FE130E04FEF5FEF6DE770E0C5
:1049A00088E290E00E949905109270064EE150E076
:1049B00066E970E015C09AE7E92E94E0F92E02E06E
:1049C0002FE130E04FEF5FEF6DE770E088E290E0BD
:1049D0000E949905C09370064EE150E068E770E0D0
:1049E00089EE95E00E94034280913A0681110FC042
:1049F000A895C09347061092240610922306C093F0
:104A000035068FE190E00E941906A89545D980915E
:104A10003A06813059F5A8958093470610922406EE
:104A200010922306809335068FE190E00E941906CC
:104A3000A89510927F0680917006813069F038F059
:104A4000823091F44EE150E06AE570E009C04EE139
:104A500050E066E970E004C04EE150E068E770E0C5
:104A600089EE95E00E940342A89513D0D0933A06B0
:104A70002FEF80E792E0215080409040E1F700C0A6
:104A800000001ECFDF91CF911F910F91FF90EF900B
:104A90000895EF92FF920F931F93CF9380917F061B
:104AA00081110C949C2E8FE190E00E9419060E94C7
:104AB000450D85E080933A06C5E080917F0681111F
:104AC0000C949C2E0E94DD0C80913A068230D9F421
:104AD00080916B068F5F80936B060FE110E02CE3F3
:104AE00030E046EE50E069E670E081E090E00E9440
:104AF000A40422E330E043EC50E068E270E088E098
:104B000090E00E94A40480913A068330D9F4809109
:104B10006B06815080936B060FE110E02CE330E0D0
:104B200046EE50E069E670E081E090E00E94A40467
:104B300022E330E043EC50E068E270E088E090E08F
:104B40000E94A40480916B068E3010F010926B06C8
:104B5000E0916B068E2F90E08E30910508F097C79C
:104B6000FC01E958FF4F80911206909113060C94B6
:104B7000F83E892B61F57AE2E72E74E0F72E01E02A
:104B80002FE130E04FEF5FEF62E370E08FE090E005
:104B90000E949905E3E2EE2EE4E0FE2E2FE130E0E4
:104BA0004FEF5FEF66E470E08CE390E00E949905C0
:104BB000E090E905F090EA0503E02FE130E04FEFE7
:104BC0005FEF62E870E080E590E00E94DF05809191
:104BD000120690911306019709F07BC65AE2E52E62
:104BE00054E0F52E01E02FE130E04FEF5FEF62E39C
:104BF00070E08FE090E00E94990563E2E62E64E0A9
:104C0000F62E2FE130E04FEF5FEF66E470E08CE3CB
:104C100090E00E949905E090E905F090EA054EC603
:104C2000892B61F53BE0E32E34E0F32E01E02FE128
:104C300030E04FEF5FEF62E370E08FE090E00E94C2
:104C400099054DEFE42E43E0F42E2FE130E04FEFD5
:104C50005FEF66E470E08CE390E00E949905E090DD
:104C6000EB05F090EC0503E02FE130E04FEF5FEF54
:104C700062E870E080E590E00E94DF058091120616
:104C8000909113068130910531F480916B068F5F0E
:104C900080936B062EC0029761F59BE0E92E94E0AD
:104CA000F92E01E02FE130E04FEF5FEF62E370E0BB
:104CB0008FE090E00E9499052DEFE22E23E0F22E86
:104CC0002FE130E04FEF5FEF66E470E08CE390E0BF
:104CD0000E949905E090EB05F090EC0503E02FE1D0
:104CE00030E04FEF5FEF62E870E080E590E00E9417
:104CF000DF058091120690911306049761F50BE091
:104D0000E02E04E0F02E01E02FE130E04FEF5FEF06
:104D100062E370E08FE090E00E9499058DEFE82E4D
:104D200083E0F82E2FE130E04FEF5FEF66E470E0B4
:104D30008CE390E00E949905E090EB05F090EC0583
:104D400003E02FE130E04FEF5FEF62E870E080E5D5
:104D500090E00E94DF05809112069091130605975E
:104D600061F5BBE0EB2EB4E0FB2E01E02FE130E07B
:104D70004FEF5FEF62E370E08FE090E00E949905F3
:104D80001DEFE12E13E0F12E2FE130E04FEF5FEF4A
:104D900066E470E08CE390E00E949905E090EB05FA
:104DA000F090EC0503E02FE130E04FEF5FEF62E8B9
:104DB00070E080E590E00E94DF05809112069091FE
:104DC0001306069709F063C6FBE0EF2EF4E0FF2E12
:104DD00001E02FE130E04FEF5FEF62E370E08FE042
:104DE00090E00E949905ADEFEA2EA3E0FA2E2FE1A4
:104DF00030E04FEF5FEF66E470E08CE390E00E94FC
:104E00009905E090EB05F090EC05D8C4892B61F58D
:104E100075EEE72E73E0F72E01E02FE130E04FEF63
:104E20005FEF62E370E08FE090E00E949905EDECA7
:104E3000EE2EE3E0FE2E2FE130E04FEF5FEF66E471
:104E400070E08FE090E00E949905E090ED05F09011
:104E5000EE0503E02FE130E04FEF5FEF62E870E036
:104E600080E590E00E94DF05809112069091130684
:104E7000019709F02EC555EEE52E53E0F52E01E021
:104E80002FE130E04FEF5FEF62E370E08FE090E002
:104E90000E9499056DECE62E63E0F62E2FE130E0DE
:104EA0004FEF5FEF66E470E08FE090E00E949905BD
:104EB000E090ED05F090EE0501C5892B61F535EB2D
:104EC000E32E33E0F32E01E02FE130E04FEF5FEF10
:104ED00062E370E08FE090E00E9499054DE9E42ED6
:104EE00043E0F42E2FE130E04FEF5FEF66E470E037
:104EF0008FE090E00E949905E090EF05F090F005BA
:104F000003E02FE130E04FEF5FEF62E870E080E513
:104F100090E00E94DF058091120690911306813087
:104F2000910531F480916B068F5F80936B062EC0E4
:104F3000029761F595EBE92E93E0F92E01E02FE160
:104F400030E04FEF5FEF62E370E08FE090E00E94AF
:104F500099052DE9E22E23E0F22E2FE130E04FEF0C
:104F60005FEF66E470E08FE090E00E949905E090CA
:104F7000EF05F090F00503E02FE130E04FEF5FEF39
:104F800062E870E080E590E00E94DF058091120603
:104F900090911306049761F505EBE02E03E0F02EE7
:104FA00001E02FE130E04FEF5FEF62E370E08FE070
:104FB00090E00E9499058DE9E82E83E0F82E2FE11C
:104FC00030E04FEF5FEF66E470E08FE090E00E942A
:104FD0009905E090EF05F090F00503E02FE130E057
:104FE0004FEF5FEF62E870E080E590E00E94DF0540
:104FF0008091120690911306059761F5B5EBEB2EA3
:10500000B3E0FB2E01E02FE130E04FEF5FEF62E312
:1050100070E08FE090E00E9499051DE9E12E13E019
:10502000F12E2FE130E04FEF5FEF66E470E08FE0AC
:1050300090E00E949905E090EF05F090F00503E004
:105040002FE130E04FEF5FEF62E870E080E590E045
:105050000E94DF058091120690911306069709F0D1
:1050600016C5F5EBEF2EF3E0FF2E01E02FE130E067
:105070004FEF5FEF62E370E08FE090E00E949905F0
:10508000ADE9EA2EA3E0FA2E2FE130E04FEF5FEF1B
:1050900066E470E08FE090E00E949905E090EF05F3
:1050A000F090F0058BC3892BC9F5E5E8EE2EE3E01F
:1050B000FE2E01E02FE130E04FEF5FEF6CE370E098
:1050C0008FE090E00E9499058091F1059091F205A2
:1050D000019779F472E4E72E75E0F72E03E02FE1F3
:1050E00030E04FEF5FEF62E870E080E590E00E9413
:1050F00099058091F1059091F205892B79F46DE382
:10510000E62E65E0F62E03E02FE130E04FEF5FEF93
:1051100062E870E080E590E00E94990580911206B7
:10512000909113060197C9F555E8E52E53E0F52E49
:1051300001E02FE130E04FEF5FEF6CE370E08FE0D4
:1051400090E00E9499058091F1059091F2050197F8
:1051500079F442E4E42E45E0F42E03E02FE130E060
:105160004FEF5FEF62E870E080E590E00E94990504
:105170008091F1059091F205892B79F43DE3E32EBE
:1051800035E0F32E03E02FE130E04FEF5FEF62E810
:1051900070E080E590E00E94990580911206909160
:1051A00013060297C9F525E8E22E23E0F22E01E06E
:1051B0002FE130E04FEF5FEF6CE370E08FE090E0C5
:1051C0000E9499058091F1059091F205019779F47B
:1051D00092E4E92E95E0F92E03E02FE130E04FEF65
:1051E0005FEF62E870E080E590E00E9499058091B1
:1051F000F1059091F205892B79F48DE3E82E85E095
:10520000F82E03E02FE130E04FEF5FEF62E870E04F
:1052100080E590E00E949905809112069091130616
:105220009C01245031092230310508F4F6C3069759
:1052300009F02DC405E8E02E03E0F02E01E02FE197
:1052400030E04FEF5FEF6CE370E08FE090E00E94A2
:1052500099058091F1059091F205019779F412E496
:10526000E12E15E0F12E03E02FE130E04FEF5FEF8C
:1052700062E870E080E590E00E9499058091F10578
:105280009091F205892B09F002C4BDE3EB2EB5E045
:10529000FB2E03E02FE130E04FEF5FEF62E870E0BC
:1052A00080E590E00E949905F2C3892B61F5FDE647
:1052B000EF2EF3E0FF2E01E02FE130E04FEF5FEF44
:1052C00062E370E08FE090E00E949905A5E5EA2E88
:1052D000A3E0FA2E2FE130E04FEF5FEF66E470E0DD
:1052E0008FE090E00E949905E090F305F090F405BE
:1052F00003E02FE130E04FEF5FEF62E870E080E520
:1053000090E00E94DF0580911206909113060197AC
:1053100061F57DE6E72E73E0F72E01E02FE130E046
:105320004FEF5FEF62E370E08FE090E00E9499053D
:10533000E5E5EE2EE3E0FE2E2FE130E04FEF5FEFEC
:1053400066E470E08FE090E00E949905E090F3053C
:10535000F090F40503E02FE130E04FEF5FEF62E8FB
:1053600070E080E590E00E94DF0580911206909148
:105370001306029761F55DE6E52E53E0F52E01E098
:105380002FE130E04FEF5FEF62E370E08FE090E0FD
:105390000E94990565E5E62E63E0F62E2FE130E0E8
:1053A0004FEF5FEF66E470E08FE090E00E949905B8
:1053B000E090F305F090F40503E02FE130E04FEFCB
:1053C0005FEF62E870E080E590E00E94DF05809189
:1053D0001206909113069C012450310922303105A8
:1053E00008F41BC3069709F052C33DE6E32E33E0F1
:1053F000F32E01E02FE130E04FEF5FEF62E370E06A
:105400008FE090E00E94990545E5E42E43E0F42EFC
:105410002FE130E04FEF5FEF66E470E08FE090E067
:105420000E949905E090F305F090F405C7C1892B1F
:1054300061F59DE3E92E93E0F92E01E02FE130E0E4
:105440004FEF5FEF62E370E08FE090E00E9499051C
:1054500025E2E22E23E0F22E2FE130E04FEF5FEF66
:1054600066E470E08FE090E00E949905E090F50519
:10547000F090F60503E02FE130E04FEF5FEF62E8D8
:1054800070E080E590E00E94DF0580911206909127
:105490001306019761F50DE3E02E03E0F02E01E025
:1054A0002FE130E04FEF5FEF62E370E08FE090E0DC
:1054B0000E94990585E2E82E83E0F82E2FE130E086
:1054C0004FEF5FEF66E470E08FE090E00E94990597
:1054D000E090F505F090F60503E02FE130E04FEFA6
:1054E0005FEF62E870E080E590E00E94DF05809168
:1054F0001206909113068230910531F480916B066B
:105500008F5F80936B062EC0049761F5BDE3EB2E91
:10551000B3E0FB2E01E02FE130E04FEF5FEF62E3FD
:1055200070E08FE090E00E94990515E2E12E13E013
:10553000F12E2FE130E04FEF5FEF66E470E08FE097
:1055400090E00E949905E090F505F090F60503E0E3
:105550002FE130E04FEF5FEF62E870E080E590E030
:105560000E94DF058091120690911306059761F560
:10557000FDE3EF2EF3E0FF2E01E02FE130E04FEFEF
:105580005FEF62E370E08FE090E00E949905A5E292
:10559000EA2EA3E0FA2E2FE130E04FEF5FEF66E452
:1055A00070E08FE090E00E949905E090F505F090A2
:1055B000F60503E02FE130E04FEF5FEF62E870E0C7
:1055C00080E590E00E94DF0580911206909113061D
:1055D00022C2892B61F57DE0E72E73E0F72E01E012
:1055E0002FE130E04FEF5FEF62E370E08FE090E09B
:1055F0000E949905E5EFEE2EE2E0FE2E2FE130E06D
:105600004FEF5FEF66E470E08FE090E00E94990555
:10561000E090F705F090F80503E02FE130E04FEF60
:105620005FEF62E870E080E590E00E94DF05809126
:105630001206909113068130910531F480916B062A
:105640008F5F80936B062EC0029761F55DE0E52EBB
:1056500053E0F52E01E02FE130E04FEF5FEF62E322
:1056600070E08FE090E00E94990565EFE62E62E021
:10567000F62E2FE130E04FEF5FEF66E470E08FE051
:1056800090E00E949905E090F705F090F80503E09E
:105690002FE130E04FEF5FEF62E870E080E590E0EF
:1056A0000E94DF058091120690911306049761F520
:1056B0003DE0E32E33E0F32E01E02FE130E04FEF49
:1056C0005FEF62E370E08FE090E00E94990545EFA4
:1056D000E42E42E0F42E2FE130E04FEF5FEF66E47E
:1056E00070E08FE090E00E949905E090F705F0905F
:1056F000F80503E02FE130E04FEF5FEF62E870E084
:1057000080E590E00E94DF058091120690911306DB
:10571000059761F59DE0E92E93E0F92E01E02FE178
:1057200030E04FEF5FEF62E370E08FE090E00E94C7
:10573000990525EFE22E22E0F22E2FE130E04FEF27
:105740005FEF66E470E08FE090E00E949905E090E2
:10575000F705F090F80503E02FE130E04FEF5FEF41
:1057600062E870E080E590E00E94DF05809112061B
:1057700090911306069709F08AC11DE0E12E13E00F
:10578000F12E01E02FE130E04FEF5FEF62E370E0D8
:105790008FE090E00E94990585EFE82E82E0F82ED8
:1057A0002FE130E04FEF5FEF66E470E08FE090E0D4
:1057B0000E949905E090F705F090F80503E02FE1CD
:1057C00030E04FEF5FEF62E870E080E590E00E942C
:1057D000DF055DC1892BF1F4B5E7EB2EB2E0FB2EBE
:1057E00001E02FE130E04FEF5FEF6CE370E08FE01E
:1057F00090E00E949905E0900106F090020603E017
:105800002FE130E04FEF5FEF62E870E080E590E07D
:105810000E94DF058091120690911306019709F00E
:1058200058C0A5E7EA2EA2E0FA2E01E02FE130E011
:105830004FEF5FEF6CE370E08FE090E00E9499051E
:10584000E0900106F090020639C0892BF1F4FBECE0
:10585000EF2EF2E0FF2E01E02FE130E04FEF5FEF9F
:105860006CE370E08FE090E00E949905E090030601
:10587000F090040603E02FE130E04FEF5FEF62E8C5
:1058800070E080E590E00E94DF0580911206909123
:1058900013060197F1F4EBECEE2EE2E0FE2E01E0B0
:1058A0002FE130E04FEF5FEF6CE370E08FE090E0CE
:1058B0000E949905E0900306F090040603E02FE1B2
:1058C00030E04FEF5FEF62E870E080E590E00E942B
:1058D000DF0580911206909113068230910509F43C
:1058E0009CC09C01245031092230310508F093C03E
:1058F00094C0892B09F07CC073EEE72E72E0F72E7E
:1059000001E02FE130E04FEF5FEF6CE370E08EE1FC
:1059100090E00E9499058091F9059091FA05019710
:1059200079F462E4E62E65E0F62E03E02FE130E044
:105930004FEF5FEF62E870E080E590E00E9499052C
:105940008091F9059091FA05892B79F45DE3E52EB4
:1059500055E0F52E03E02FE130E04FEF5FEF62E816
:1059600070E080E590E00E9499058091F9058093B0
:10597000D8053EC0892BE1F58091D80581110AC078
:1059800010926B0643C0892B99F58091D80581113F
:10599000AEC1F6CF8130D1F53DE6E32E33E0F32EF4
:1059A00001E02FE130E04FEF5FEF62E370E08FE066
:1059B00090E00E94990545EBE42E42E0F42E2FE1A1
:1059C00030E04FEF5FEF66E470E08FE090E00E9420
:1059D0009905E090FB05F090FC0503E02FE130E035
:1059E0004FEF5FEF62E870E080E590E00E94DF0536
:1059F00080911206909113068130910571F08230EA
:105A0000910559F08430910541F002C080E090E0AA
:105A10008530910511F00697D1F580916B068F5F67
:105A200080936B0634C0009731F09C0121503109FE
:105A30002230310518F410926B0620C00497F1F45F
:105A40008EE4E82E82E0F82E01E02FE130E04FEF07
:105A50005FEF6CE370E08FE090E00E949905E090CA
:105A60000506F090060603E02FE130E04FEF5FEF10
:105A700062E870E080E590E00E94DF058091120608
:105A8000909113060597029710F410926B0680917F
:105A90003A06813009F00EC180937F0610924706C6
:105AA0008091120690911306892B41F5E0911D0615
:105AB000F0911E06E830F10508F5EB57FF4F4EE177
:105AC00050E00C94F83E64E972E014C066E772E0BE
:105AD00011C068E572E00EC06AE372E00BC06CE1D1
:105AE00072E008C06EEF71E005C060EE71E002C0C8
:105AF00062EC71E089EE95E00E94204280911206EE
:105B0000909113060197E1F480911D0690911E0675
:105B10008130910569F038F0029791F44EE150E040
:105B200068E671E009C04EE150E064EA71E004C04B
:105B30004EE150E066E871E089EE95E00E94204277
:105B400080911206909113060297E1F480911D0650
:105B500090911E068130910569F038F0029791F41A
:105B60004EE150E06EE071E009C04EE150E06AE4C1
:105B700071E004C04EE150E06CE271E089EE95E026
:105B80000E94204280911206909113060497E1F43E
:105B900080911D0690911E068130910569F038F0C4
:105BA000029791F44EE150E064EB70E009C04EE1E1
:105BB00050E060EF70E004C04EE150E062ED70E054
:105BC00089EE95E00E942042809112069091130682
:105BD0000597E1F480911D0690911E068130910594
:105BE00069F038F0029791F44EE150E06AE570E018
:105BF00009C04EE150E066E970E004C04EE150E0BB
:105C000068E770E089EE95E00E94204280911206DC
:105C1000909113060697E1F480911D0690911E065F
:105C20008130910569F038F0029791F44EE150E02F
:105C300060E070E009C04EE150E06CE370E004C049
:105C40004EE150E06EE170E089EE95E00E94204266
:105C50008FE190E00E941906809112069091130640
:105C6000892B09F477D18091120690911306019740
:105C700011F40E946A3880911206909113060297DF
:105C800011F40E94713980911206909113060497C5
:105C900011F40E94763A80911206909113060597AE
:105CA00011F40E94432480911206909113060697E6
:105CB00009F448D080913A0681110CC081E08093AC
:105CC0007F0610924706109207068FE190E00E942F
:105CD0001906E3D2C0933A062FE788E391E02150FA
:105CE00080409040E1F700C000000C945D258130B9
:105CF00009F08CCE9EE9E92E92E0F92E01E02FE129
:105D000030E04FEF5FEF62E370E08FE090E00E94E1
:105D100099052BE8E22E22E0F22E2FE130E04FEF42
:105D20005FEF66E470E08FE090E00E949905E090FC
:105D3000FD05F090FE0551CECF911F910F91FF9080
:105D4000EF900895EF92FF920F931F93CF93DF93FD
:105D5000A895809147068111F6C08FE190E00E94DE
:105D600019060E944F0C80916D0690E090931E06DC
:105D700080931D0685E080933A06C1E0D5E08091CE
:105D800047068111E0C0A8950E94DD0C80913A067B
:105D90008230A9F480911D0690911E060196909381
:105DA0001E0680931D060FE110E02CE330E046EE66
:105DB00050E069E670E081E090E00E94A4048091E8
:105DC0003A068330A9F480911D0690911E06019732
:105DD00090931E0680931D060FE110E02CE330E047
:105DE00046EE50E069E670E081E090E00E94A40495
:105DF00080911D0690911E06039720F010921E06BA
:105E000010921D0680911D0690911E06813091050D
:105E100089F1D0F0029709F046C080E7E82E84E0CF
:105E2000F82E02E02FE130E04FEF5FEF6DE770E01A
:105E300088E290E00E94990582E080936D064EE131
:105E400050E060E070E02BC024E8E22E24E0F22E67
:105E500002E02FE130E04FEF5FEF6DE770E088E2A6
:105E600090E00E94990510926D064EE150E06CE3BF
:105E700070E015C09AE7E92E94E0F92E02E02FE1D8
:105E800030E04FEF5FEF6DE770E088E290E00E9456
:105E90009905C0936D064EE150E06EE170E089EE29
:105EA00095E00E94034280913A06811110C0A895A6
:105EB000C09347061092240610922306C09335061D
:105EC0008FE190E00E941906A8950E944C1E8091D7
:105ED0003A06813061F5A895809347061092240612
:105EE00010922306809335068FE190E00E941906F8
:105EF000A89510927F0680916D06813069F038F088
:105F0000823091F44EE150E060E070E009C04EE173
:105F100050E06CE370E004C04EE150E06EE170E0F0
:105F200089EE95E00E940342A8950E944925D093EE
:105F30003A062FEF80E792E0215080409040E1F751
:105F400000C000001CCFDF91CF911F910F91FF90F7
:105F5000EF900895AF92BF92CF92DF92EF92FF92AF
:105F60000F931F93CF93DF93A895809147068111DC
:105F700089C18FE190E00E9419060E944F0C809128
:105F8000710690E090931E0680931D0685E0809335
:105F90003A06E7E0DE2EF6E0CF2ED5E0A4E0BA2EFA
:105FA000B3E0AB2EC1E08091470681116BC1A8958B
:105FB0000E94DD0C80913A068230A9F480911D0682
:105FC00090911E06019690931E0680931D060FE188
:105FD00010E02CE330E046EE50E069E670E081E04E
:105FE00090E00E94A40480913A068330A9F4809145
:105FF0001D0690911E06019790931E0680931D0624
:106000000FE110E02CE330E046EE50E069E670E08E
:1060100081E090E00E94A40480911D0690911E06EC
:10602000089720F010921E0610921D06E0911D06A2
:10603000F0911E06E830F10508F0BEC0E357FF4FAF
:106040000C94F83E73E9E72E74E0F72E02E02FE19E
:1060500030E04FEF5FEF6DE770E082E390E00E9489
:106060009905109271064EE150E064E972E09AC021
:106070006EE8E62E64E0F62E02E02FE130E04FEF0E
:106080005FEF6DE770E082E390E00E949905C093B6
:1060900071064EE150E066E772E084C054E8E52EF8
:1060A00054E0F52E02E02FE130E04FEF5FEF6DE7B7
:1060B00070E088E290E00E94990582E0809371068A
:1060C0004EE150E068E572E06DC04AE7E42E44E03E
:1060D000F42E02E02FE130E04FEF5FEF6DE770E06C
:1060E00088E290E00E949905A09271064EE150E08E
:1060F0006AE372E057C030E7E32E34E0F32E02E0AB
:106100002FE130E04FEF5FEF6DE770E088E290E065
:106110000E949905B092710644E150E06CE172E092
:1061200041C026E6E22E24E0F22E02E02FE130E02C
:106130004FEF5FEF6DE770E088E290E00E94990515
:10614000D09371064EE150E06EEF71E02BC09CE5FC
:10615000E92E94E0F92E02E02FE130E04FEF5FEFFF
:106160006DE770E088E290E00E949905C0927106A8
:106170004EE150E060EE71E015C082E5E82E84E06B
:10618000F82E02E02FE130E04FEF5FEF6DE770E0B7
:1061900088E290E00E949905D09271064EE150E0AD
:1061A00062EC71E089EE95E00E9403428FE59AEE81
:1061B0000197F1F700C0000080913A0681110FC0ED
:1061C000A895C09347061092240610922306C09308
:1061D00035068FE190E00E9419060E944C1E8091C6
:1061E0003A06813009F041C0A89580934706109285
:1061F000240610922306809335068FE190E00E94DA
:10620000190610927F06E09171068E2F90E088307B
:10621000910540F5FC01EB56FF4F4EE150E00C9428
:10622000F83E64E972E014C066E772E011C068E508
:1062300072E00EC06AE372E00BC06CE172E008C06D
:106240006EEF71E005C060EE71E002C062EC71E0DB
:1062500089EE95E00E9403428FE59AEE0197F1F7EF
:1062600000C00000A8950E944925D0933A06A89541
:106270009FEF20E782E0915020408040E1F700C08E
:10628000000091CEDF91CF911F910F91FF90EF9081
:10629000DF90CF90BF90AF900895BF92CF92DF92E2
:1062A000EF92FF920F931F93CF93DF938091070696
:1062B000811106C78FE190E00E9419060E94450DEA
:1062C00010926C0685E080933A0698E5C92E92E01C
:1062D000D92ECAE5D0E025E0B22E809107068111C3
:1062E000EFC6E0916B068E2F90E08E30910508F09E
:1062F000D6C6FC01E356FF4F0C94F83E1AE2E12E9D
:1063000014E0F12E01E02FE130E04FEF5FEF62E3A8
:1063100070E08FE090E00E94990583E2E82E84E02F
:10632000F82E2FE130E04FEF5FEF66E470E08CE392
:1063300090E00E949905E090E905F090EA0503E0FD
:106340002FE130E040E058EF62E870E080E590E057
:106350000E94DF058091E9059091EA059093DD05A3
:106360008093DC050E94DD0C80913A068230A9F40E
:106370008091DC059091DD0501969093DD05809379
:10638000DC050FE110E02CE330E046EE50E069E67A
:1063900070E081E090E00E94A40480913A0683308E
:1063A000A9F48091DC059091DD0501979093DD05BE
:1063B0008093DC050FE110E02CE330E046EE50E086
:1063C00069E670E081E090E00E94A4048091DC0521
:1063D0009091DD058F35914020F01092DD051092EF
:1063E000DC058091DC059091DD059093EA058093B2
:1063F000E9054CC6ABE0EA2EA4E0FA2E01E02FE15D
:1064000030E04FEF5FEF62E370E08FE090E00E94DA
:106410009905BDEFEB2EB3E0FB2E2FE130E04FEFFF
:106420005FEF66E470E08CE390E00E949905E090F5
:10643000EB05F090EC0503E02FE130E040E058EF91
:1064400062E870E080E590E00E94DF058091EB0556
:106450009091EC0590933206809331060E94DD0CFA
:1064600080913A068230A9F48091310690913206EB
:10647000019690933206809331060FE110E02CE3F1
:1064800030E046EE50E069E670E081E090E00E9486
:10649000A40480913A068330A9F48091310690914A
:1064A0003206019790933206809331060FE110E097
:1064B0002CE330E046EE50E069E670E081E090E0E9
:1064C0000E94A4048091310690913206853F91404C
:1064D00020F0109232061092310680913106909190
:1064E00032069093EC058093EB05D0C5E5EEEE2ED9
:1064F000E3E0FE2E01E02FE130E04FEF5FEF62E3DB
:1065000070E08FE090E00E949905FDECEF2EF3E043
:10651000FF2E2FE130E04FEF5FEF66E470E08FE099
:1065200090E00E949905E090ED05F090EE0503E003
:106530002FE130E040E058EF62E870E080E590E065
:106540000E94DF058091ED059091EE0590937A060B
:10655000809379060E94DD0C80913A068230A9F47E
:106560008091790690917A06019690937A068093AD
:1065700079060FE110E02CE330E046EE50E069E6EA
:1065800070E081E090E00E94A40480913A0683309C
:10659000A9F48091790690917A06019790937A06F2
:1065A000809379060FE110E02CE330E046EE50E0F6
:1065B00069E670E081E090E00E94A4048091790691
:1065C00090917A064F9730F08FE090E090937A06A2
:1065D000809379068091790690917A060F9730F42E
:1065E0008FE090E090937A06809379068091790607
:1065F00090917A069093EE058093ED0547C565EB83
:10660000E62E63E0F62E01E02FE130E04FEF5FEF82
:1066100062E370E08FE090E00E9499057DE9E72E4B
:1066200073E0F72E2FE130E04FEF5FEF66E470E0AC
:106630008FE090E00E949905E090EF05F090F00562
:1066400003E02FE130E040E058EF62E870E080E5E1
:1066500090E00E94DF058091EF059091F005909306
:106660001A06809319060E94DD0C80913A0682304A
:10667000A9F48091190690911A06019690931A0632
:10668000809319060FE110E02CE330E046EE50E075
:1066900069E670E081E090E00E94A40480913A06EF
:1066A0008330A9F48091190690911A06019790936E
:1066B0001A06809319060FE110E02CE330E046EE55
:1066C00050E069E670E081E090E00E94A4048091CF
:1066D000190690911A064F9730F08FE090E0909352
:1066E0001A06809319068091190690911A060F9741
:1066F00030F48FE090E090931A0680931906809111
:10670000190690911A069093F0058093EF05BEC488
:1067100055E8E52E53E0F52E01E02FE130E04FEF94
:106720005FEF6CE370E08FE090E00E94990580914C
:10673000F1059091F205019779F442E4E42E45E0E9
:10674000F42E03E02FE130E040E058EF62E870E023
:1067500080E590E00E9499058091F1059091F20505
:10676000892B79F43DE3E32E35E0F32E03E02FE1AE
:1067700030E040E058EF62E870E080E590E00E9491
:1067800099058091F105809346060E94DD0C809169
:106790003A06823089F4809146068F5F80934606E0
:1067A0000FE110E02CE330E046EE50E069E670E0E7
:1067B00081E090E00E94A40480913A06833089F43D
:1067C000809146068150809346060FE110E02CE34D
:1067D00030E046EE50E069E670E081E090E00E9433
:1067E000A40480914606823010F0109246068091F3
:1067F000460690E09093F2058093F10547C49DE62C
:10680000E92E93E0F92E01E02FE130E04FEF5FEF4A
:1068100062E370E08FE090E00E94990525E5E22EAA
:1068200023E0F22E2FE130E04FEF5FEF66E470E0FF
:106830008FE090E00E949905E090F305F090F40558
:1068400003E020E038EF4FEF5FEF62E870E080E5B3
:1068500090E00E94DF058091F3059091F4059093FC
:106860001806809317060E94DD0C80913A0682304C
:10687000A9F4809117069091180601969093180636
:10688000809317060FE110E02CE330E046EE50E075
:1068900069E670E081E090E00E94A40480913A06ED
:1068A0008330A9F480911706909118060197909370
:1068B0001806809317060FE110E02CE330E046EE57
:1068C00050E069E670E081E090E00E94A4048091CD
:1068D0001706909118068B3F910520F0109218062C
:1068E0001092170680911706909118069093F40560
:1068F0008093F305CBC31DE3E12E13E0F12E01E0FD
:106900002FE130E04FEF5FEF62E370E08FE090E067
:106910000E94990585E2E82E83E0F82E2FE130E011
:106920004FEF5FEF66E470E08FE090E00E94990522
:10693000E090F505F090F60503E02FE130E040E04F
:1069400058EF62E870E080E590E00E94DF058091FA
:10695000F5059091F60590932A06809329060E94EA
:10696000DD0C80913A068230A9F48091290690913D
:106970002A06019690932A06809329060FE110E0DB
:106980002CE330E046EE50E069E670E081E090E014
:106990000E94A40480913A068330A9F480912906CC
:1069A00090912A06019790932A06809329060FE179
:1069B00010E02CE330E046EE50E069E670E081E064
:1069C00090E00E94A4048091290690912A068536C1
:1069D000910520F010922A0610922906809129062E
:1069E00090912A069093F6058093F5054FC3ADE08C
:1069F000EA2EA3E0FA2E01E02FE130E04FEF5FEF47
:106A000062E370E08FE090E00E949905B5EFEB2E15
:106A1000B2E0FB2E2FE130E04FEF5FEF66E470E075
:106A20008FE090E00E949905E090F705F090F8055E
:106A300003E02FE130E040E058EF62E870E080E5ED
:106A400090E00E94DF058091F7059091F805909302
:106A50002806809327060E94DD0C80913A0682303A
:106A6000A9F4809127069091280601969093280614
:106A7000809327060FE110E02CE330E046EE50E073
:106A800069E670E081E090E00E94A40480913A06FB
:106A90008330A9F48091270690912806019790935E
:106AA0002806809327060FE110E02CE330E046EE45
:106AB00050E069E670E081E090E00E94A4048091DB
:106AC0002706909128068536910520F01092280619
:106AD0001092270680912706909128069093F8053A
:106AE0008093F705D3C2F5E7EF2EF2E0FF2E01E029
:106AF0002FE130E04FEF5FEF6CE370E08FE090E06C
:106B00000E949905E0900106F090020603E02FE153
:106B100030E040E058EF62E870E080E590E00E94ED
:106B2000DF0580910106909102069093680680939C
:106B300067060E94DD0C80913A068230A9F48091AC
:106B400067069091680601969093680680936706A1
:106B50000FE110E02CE330E046EE50E069E670E033
:106B600081E090E00E94A40480913A068330A9F469
:106B700080916706909168060197909368068093CC
:106B800067060FE110E02CE330E046EE50E069E6E6
:106B900070E081E090E00E94A404809167069091EB
:106BA0006806893C910520F0D0936806C09367067B
:106BB00080916706909168068A35910520F4D093FC
:106BC0006806C09367068091670690916806909367
:106BD0000206809301065AC2EBECEE2EE2E0FE2E96
:106BE00001E02FE130E04FEF5FEF6CE370E08FE00A
:106BF00090E00E949905E0900306F090040603E0FF
:106C00002FE130E040E058EF62E870E080E590E08E
:106C10000E94DF0580910306909104069093E80599
:106C20008093E7050E94DD0C80913A068230A9F43A
:106C30008091E7059091E80501969093E80580938F
:106C4000E7050FE110E02CE330E046EE50E069E6A6
:106C500070E081E090E00E94A40480913A068330C5
:106C6000A9F48091E7059091E80501979093E805D4
:106C70008093E7050FE110E02CE330E046EE50E0B2
:106C800069E670E081E090E00E94A4048091E7054D
:106C90009091E805C39720F01092E8051092E7055F
:106CA0008091E7059091E805909304068093030690
:106CB000EDC173EEE72E72E0F72E01E02FE130E038
:106CC0004FEF5FEF6CE370E08EE190E00E9499057A
:106CD0008091F9059091FA05019779F462E4E62E26
:106CE00065E0F62E03E02FE130E040E058EF62E887
:106CF00070E080E590E00E9499058091F9059091FF
:106D0000FA05892B79F45DE3E52E55E0F52E03E0D5
:106D10002FE130E040E058EF62E870E080E590E07D
:106D20000E9499058091F9058093D8050E94DD0C99
:106D300080913A06823089F48091D8058F5F8093E4
:106D4000D8050FE110E02CE330E046EE50E069E6B4
:106D500070E081E090E00E94A40480913A068330C4
:106D600089F48091D80581508093D8050FE110E017
:106D70002CE330E046EE50E069E670E081E090E020
:106D80000E94A4048091D805823010F01092D8059A
:106D90008091D80590E09093FA058093F90576C12B
:106DA0008091D805811103C010926B0678C18130A3
:106DB00009F075C13DE6E32E33E0F32E01E02FE14B
:106DC00030E04FEF5FEF62E370E08FE090E00E9411
:106DD000990545EBE42E42E0F42E2FE130E04FEF31
:106DE0005FEF66E470E08FE090E00E949905E0902C
:106DF000FB05F090FC0503E02FE130E040E058EFA8
:106E000062E870E080E590E00E94DF058091FB057C
:106E10009091FC0590936A06809369060E94DD0CB0
:106E200080913A068230A9F48091690690916A06B1
:106E3000019690936A06809369060FE110E02CE3B7
:106E400030E046EE50E069E670E081E090E00E94BC
:106E5000A40480913A068330A9F480916906909148
:106E60006A06019790936A06809369060FE110E025
:106E70002CE330E046EE50E069E670E081E090E01F
:106E80000E94A4048091690690916A068B3F910547
:106E900020F010926A06109269068091690690911E
:106EA0006A069093FC058093FB05F0C08091D8059D
:106EB000882309F479CF813009F0F1C09EE9E92EE9
:106EC00092E0F92E01E02FE130E04FEF5FEF62E357
:106ED00070E08FE090E00E9499052BE8E22E22E01E
:106EE000F22E2FE130E04FEF5FEF66E470E08FE0CD
:106EF00090E00E949905E090FD05F090FE0503E00A
:106F00002FE130E040E058EF62E870E080E590E08B
:106F10000E94DF058091FD059091FE059093450646
:106F2000809344060E94DD0C80913A068230A9F4D9
:106F30008091440690914506019690934506809372
:106F400044060FE110E02CE330E046EE50E069E645
:106F500070E081E090E00E94A40480913A068330C2
:106F6000A9F48091440690914506019790934506B7
:106F7000809344060FE110E02CE330E046EE50E051
:106F800069E670E081E090E00E94A40480914406EC
:106F900090914506C39720F0109245061092440642
:106FA00080914406909145069093FE058093FD05DF
:106FB0006DC08EE4E82E82E0F82E01E02FE130E093
:106FC0004FEF5FEF6CE370E08FE090E00E94990577
:106FD000E0900506F090060603E02FE130E040E087
:106FE00058EF62E870E080E590E00E94DF05809154
:106FF00005069091060690930D0680930C060E945C
:10700000DD0C80913A068230A9F480910C069091B3
:107010000D06019690930D0680930C060FE110E08B
:107020002CE330E046EE50E069E670E081E090E06D
:107030000E94A40480913A068330A9F480910C0642
:1070400090910D06019790930D0680930C060FE129
:1070500010E02CE330E046EE50E069E670E081E0BD
:1070600090E00E94A4048091E7059091E80589359D
:10707000924020F0D0920D06C0920C0680910C0632
:1070800090910D0690930606809305068FE798E38E
:1070900021E0815090402040E1F700C00000809145
:1070A0003A06813051F48093070610927F068FE1F3
:1070B00090E00E9419060E944925B0923A060DC937
:1070C000DF91CF911F910F91FF90EF90DF90CF90C4
:1070D000BF900895EF92FF920F931F93CF93DF938A
:1070E000A895809147068111F5C08FE190E00E943C
:1070F00019060E944F0C80911B0690E090931E068B
:1071000080931D0685E080933A06C1E0D5E080912A
:1071100047068111DFC0A8950E94DD0C80913A06D8
:107120008230A9F480911D0690911E0601969093DD
:107130001E0680931D060FE110E02CE330E046EEC2
:1071400050E069E670E081E090E00E94A404809144
:107150003A068330A9F480911D0690911E0601978E
:1071600090931E0680931D060FE110E02CE330E0A3
:1071700046EE50E069E670E081E090E00E94A404F1
:1071800080911D0690911E06039720F010921E0616
:1071900010921D06A89580911D0690911E068130C3
:1071A000910589F1D0F0029709F046C080E7E82EFA
:1071B00084E0F82E02E02FE130E04FEF5FEF6DE763
:1071C00070E088E290E00E94990582E080931B06BF
:1071D0004EE150E068E671E02BC024E8E22E24E0A6
:1071E000F22E02E02FE130E04FEF5FEF6DE770E04D
:1071F00088E290E00E94990510921B064EE150E053
:1072000064EA71E015C09AE7E92E94E0F92E02E0F5
:107210002FE130E04FEF5FEF6DE770E088E290E044
:107220000E949905C0931B064EE150E066E871E0AC
:1072300089EE95E00E94034280913A0681110FC0C9
:10724000A895C09347061092240610922306C09377
:1072500035068FE190E00E9419060E944C1E809135
:107260003A06813059F5A895809347061092240676
:1072700010922306809335068FE190E00E94190654
:1072800010927F0680911B06813069F038F08230C1
:1072900091F44EE150E068E671E009C04EE150E043
:1072A00064EA71E004C04EE150E066E871E089EE06
:1072B00095E00E940342A8950E944925D0933A0682
:1072C0002FEF80E792E0215080409040E1F700C02E
:1072D00000001DCFDF91CF911F910F91FF90EF9094
:1072E0000895EF92FF920F931F93CF93DF93A8958A
:1072F000809147068111F3C08FE190E00E9419064A
:107300000E944F0C8091220690E090931E0680937D
:107310001D0685E080933A06C1E0D5E080914706DE
:107320008111DDC0A8950E94DD0C80913A06823063
:10733000A9F480911D0690911E06019690931E0659
:1073400080931D060FE110E02CE330E046EE50E0A4
:1073500069E670E081E090E00E94A40480913A0622
:107360008330A9F480911D0690911E060197909399
:107370001E0680931D060FE110E02CE330E046EE80
:1073800050E069E670E081E090E00E94A404809102
:107390001D0690911E06039720F010921E06109273
:1073A0001D0680911D0690911E068130910589F180
:1073B000D0F0029709F045C080E7E82E84E0F82E6F
:1073C00002E02FE130E04FEF5FEF6DE770E088E221
:1073D00090E00E94990582E0809322064EE150E001
:1073E0006EE071E02BC024E8E22E24E0F22E02E0F1
:1073F0002FE130E04FEF5FEF6DE770E088E290E063
:107400000E949905109222064EE150E06AE471E074
:1074100015C09AE7E92E94E0F92E02E02FE130E062
:107420004FEF5FEF6DE770E088E290E00E94990512
:10743000C09322064EE150E06CE271E089EE95E0E7
:10744000E2D780913A06811110C0A895C0934706F3
:107450001092240610922306C09335068FE190E027
:107460000E941906A8950E944C1E80913A06813010
:1074700051F5A89580934706109224061092230692
:10748000809335068FE190E00E94190610927F06E6
:1074900080912206813069F038F0823089F44EE123
:1074A00050E06EE071E009C04EE150E06AE471E046
:1074B00004C04EE150E06CE271E089EE95E0A3D7A4
:1074C000A8950E944925D0933A062FEF80E792E0D5
:1074D000215080409040E1F700C000001FCFDF91B5
:1074E000CF911F910F91FF90EF900895EF92FF922F
:1074F0000F931F93CF93DF93A89580914706811137
:10750000F4C08FE190E00E9419060E944F0C809118
:107510007C0690E090931E0680931D0685E0809384
:107520003A06C1E0D5E0809147068111DEC0A895FA
:107530000E94DD0C80913A068230A9F480911D06EC
:1075400090911E06019690931E0680931D060FE1F2
:1075500010E02CE330E046EE50E069E670E081E0B8
:1075600090E00E94A40480913A068330A9F48091AF
:107570001D0690911E06019790931E0680931D068E
:107580000FE110E02CE330E046EE50E069E670E0F9
:1075900081E090E00E94A40480911D0690911E0657
:1075A000039720F010921E0610921D0680911D0672
:1075B00090911E068130910589F1D0F0029709F073
:1075C00045C080E7E82E84E0F82E02E02FE130E0AD
:1075D0004FEF5FEF6DE770E088E290E00E94990561
:1075E00082E080937C064EE150E064EB70E02BC0BB
:1075F00024E8E22E24E0F22E02E02FE130E04FEF0B
:107600005FEF6DE770E088E290E00E9499051092CC
:107610007C064EE150E060EF70E015C09AE7E92E7D
:1076200094E0F92E02E02FE130E04FEF5FEF6DE7DD
:1076300070E088E290E00E949905C0937C064EE1DC
:1076400050E062ED70E089EE95E0DDD680913A067B
:10765000811110C0A895C09347061092240610927D
:107660002306C09335068FE190E00E941906A89585
:107670000E944C1E80913A06813059F5A89580935E
:1076800047061092240610922306809335068FE158
:1076900090E00E941906A89510927F0680917C06C2
:1076A000813069F038F0823089F44EE150E064EBCB
:1076B00070E009C04EE150E060EF70E004C04EE1C0
:1076C00050E062ED70E089EE95E09DD6A8950E94AD
:1076D0004925D0933A062FEF80E792E02150804071
:1076E0009040E1F700C000001ECFDF91CF911F91C5
:1076F0000F91FF90EF9008951F920F920FB60F9287
:1077000011248F939F938CB190E090937406809393
:1077100073069F918F910F900FBE0F901F90189539
:107720001F920F920FB60F9211242F938F939F9356
:107730008091E3059091E4050196883E23E092074D
:1077400028F49093E4058093E30504C01092E405C7
:107750001092E30580910E06811105C01092760605
:10776000109275060BC0813049F480917506909196
:1077700076060196909376068093750680912F0683
:10778000811105C01092E2051092E1050BC0813015
:1077900049F48091E1059091E20501969093E2050C
:1077A0008093E10580912506811105C01092E605C0
:1077B0001092E5050BC0813049F48091E505909168
:1077C000E60501969093E6058093E5059F918F91DC
:1077D0002F910F900FBE0F901F9018952FEF89E6F5
:1077E00098E1215080409040E1F700C000008FEF09
:1077F0008ABB81BB8093610081E084BB88EA8FBD36
:107800008CE08EBD1DBC1CBC17BC16BC8AE78BBDB2
:1078100082E18ABD19BC18BC1092790010927800E0
:10782000C0E1C7BF10BE87E683BF12BE11BE81E8AC
:1078300080938B0085E080938A00109289001092DB
:1078400088001092810010928000109287001092A0
:10785000860010928500109284001092830010928E
:1078600082001BB888E98AB986E08093950010925F
:1078700090008FE289B98FE181BD8FE081BD08D191
:1078800081E00E94B0038FE190E00E94190681E040
:1078900090E09093110680931006109224061092A7
:1078A000230610921306109212061092E40510920D
:1078B000E30510922C0610922B061092E005109210
:1078C0000F06109277061092080680E590E09093DC
:1078D000740680937306809164008E7F80936400A9
:1078E000809165008160809365007894A49AC5BBFF
:1078F0002FEF85EA9EE0215080409040E1F700C0E4
:10790000000015BA82EB92E08ED5813079F00E94AA
:107910005019A8950E94BD1CA89561E083EB92E0E8
:1079200098D5A89561E082EB92E093D5C1E0D0E0D4
:10793000A8958091100690911106019721F4A895C1
:107940000E944C1EA895A895809110069091110652
:10795000892B71F780917306909174068335910598
:1079600099F5D0931106C09310060E946E130FE193
:1079700010E02CE330E044E650E06BE470E08EE68B
:1079800090E00E94A40424E230E04AE550E064E67E
:1079900070E088E090E00E94A40424E230E04AE530
:1079A00050E064E670E088E090E00E94A40424E2E5
:1079B00030E04AE550E064E670E08FED90E00E9430
:1079C000A4040E944C1EA8950E94301D0E948F1393
:1079D000A89503E02FE130E04FEF5FEF69E170E041
:1079E00085E890E00E94E3100E94DE1C0E94821055
:1079F0008091100690911106019781F5A8950E943B
:107A00006E130FE110E02CE330E044E650E06BE44D
:107A100070E08EE690E00E94A40424E230E04AE5A3
:107A200050E064E670E088E090E00E94A40424E264
:107A300030E04AE550E064E670E088E090E00E94C3
:107A4000A40424E230E04AE550E064E670E08FED03
:107A500090E00E94A4040E944C1EA8952FEF81EE96
:107A600094E0215080409040E1F700C000000E9467
:107A7000D20E0E94071D0E94580F0E94C80F58CFB7
:107A8000C098AB9AAF9A8FB9779BFECF8FB108950C
:107A900087E087BBC09AAB9AAF9A83E58DB91EB8D1
:107AA00080E8EEDF80E0ECDF80E0EADF8AE18A95C3
:107AB000F1F700C00895EF92FF920F931F93CF93B9
:107AC000DF9300D000D0CDB7DEB77C018B01A89545
:107AD000AB9AAF9A1C821B821A82198280EDD0DF8A
:107AE00080E0CEDF8FB190E09C838B838B819C8183
:107AF000982F88279C838B8380E0C2DF2FB18B81F6
:107B00009C81822B9C838B838B819C8133E0969517
:107B100087953A95E1F79C838B8387EC90E00197FA
:107B2000F1F700C0000080E9ABDF80E0A9DF8FB192
:107B300090E09A83898389819A81982F88279A83F4
:107B4000898380E09DDF2FB189819A81822B9A837E
:107B5000898389819A8153E0969587955A95E1F7B3
:107B60009A8389838B819C81F701918380838981AA
:107B70009A81F801918380830F900F900F900F905E
:107B8000DF91CF911F910F91FF90EF90089570D0EA
:107B900088F09F5790F0B92F9927B751A0F0D1F0F6
:107BA000660F771F881F991F1AF0BA95C9F712C080
:107BB000B13081F077D0B1E0089574C0672F782F8D
:107BC0008827B85F39F0B93FCCF3869577956795EC
:107BD000B395D9F73EF490958095709561957F4F58
:107BE0008F4F9F4F0895E89409C097FB3EF49095FE
:107BF0008095709561957F4F8F4F9F4F9923A9F086
:107C0000F92F96E9BB279395F69587957795679514
:107C1000B795F111F8CFFAF4BB0F11F460FF1BC058
:107C20006F5F7F4F8F4F9F4F16C0882311F096E9EB
:107C300011C0772321F09EE8872F762F05C0662399
:107C400071F096E8862F70E060E02AF09A95660F52
:107C5000771F881FDAF7880F9695879597F908950B
:107C600057FD9058440F551F59F05F3F71F04795ED
:107C7000880F97FB991F61F09F3F79F087950895D2
:107C8000121613061406551FF2CF4695F1DF08C0F1
:107C9000161617061806991FF1CF8695710561050E
:107CA00008940895E894BB2766277727CB0197F9B6
:107CB00008950BD078C069D028F06ED018F09523C5
:107CC00009F05AC05FC01124EECFCADFA0F3959F20
:107CD000D1F3950F50E0551F629FF001729FBB27B3
:107CE000F00DB11D639FAA27F00DB11DAA1F649F5F
:107CF0006627B00DA11D661F829F2227B00DA11D12
:107D0000621F739FB00DA11D621F839FA00D611D97
:107D1000221F749F3327A00D611D231F849F600DB8
:107D2000211D822F762F6A2F11249F5750408AF0F1
:107D3000E1F088234AF0EE0FFF1FBB1F661F771F7D
:107D4000881F91505040A9F79E3F510570F014C014
:107D5000AACF5F3FECF3983EDCF386957795679565
:107D6000B795F795E7959F5FC1F7FE2B880F911D9B
:107D70009695879597F9089597F99F6780E870E041
:107D800060E008959FEF80EC089500240A94161691
:107D9000170618060906089500240A9412161306F9
:107DA000140605060895092E0394000C11F4882387
:107DB00052F0BB0F40F4BF2B11F460FF04C06F5FA3
:107DC0007F4F8F4F9F4F0895AA1BBB1B51E107C0E8
:107DD000AA1FBB1FA617B70710F0A61BB70B881F5B
:107DE000991F5A95A9F780959095BC01CD010895EA
:107DF000EE0FFF1F0024001C0BBE0790F691E02D34
:107E00000994A29FB001B39FC001A39F700D811D73
:107E10001124911DB29F700D811D1124911D089593
:107E2000BB274A3031F4992322F4BDE29095819525
:107E30009F4F01C0BB27FB015527AA27880F991F19
:107E4000AA1FA41710F0A41B83955051B9F7A05D89
:107E5000AA3308F0A95DA193009779F7B111B19306
:107E60001192CB0126C2CF93DF93CDB7DEB7AE011F
:107E70004B5F5F4FFA0161917191AF018091820672
:107E80009091830603D0DF91CF9108952F923F9276
:107E90004F925F926F927F928F929F92AF92BF921A
:107EA000CF92DF92EF92FF920F931F93CF93DF93C6
:107EB000CDB7DEB72B970FB6F894DEBF0FBECDBFA0
:107EC0006C017B018A01FC0117821682838181FF8C
:107ED000BFC1CE0101963C01F6019381F70193FDEC
:107EE000859193FF81917F01882309F4ADC185328B
:107EF00039F493FD859193FF81917F01853221F4BF
:107F0000B60190E0E6D1E8CF912C212C312CFFE195
:107F1000F315D8F08B3279F038F4803279F083326F
:107F2000A1F4232D20611DC08D3261F0803369F4EE
:107F3000232D216016C0832D8260382EE32DE4604E
:107F40003E2E2AC0F32DF8601DC037FC2DC020ED59
:107F5000280F2A3040F08E32B9F436FC75C1232D3B
:107F60002064322E19C036FE06C08AE0989E200D8D
:107F70001124922E11C0EAE02E9E200D1124222EF3
:107F8000F32DF0623F2E08C08C3621F4832D8068DB
:107F9000382E02C0883641F4F70193FD859193FF96
:107FA00081917F018111B3CF982F9F7D955493309C
:107FB00028F40C5F1F4F9FE399830DC0833631F087
:107FC000833771F0833509F055C020C0F8018081F6
:107FD00089830E5F1F4F88248394912C530112C014
:107FE0002801F2E04F0E511CF801A080B18036FE4E
:107FF00003C0692D70E002C06FEF7FEFC5014ED165
:108000004C018201F32DFF773F2E15C0280122E09D
:10801000420E511CF801A080B18036FE03C0692DCC
:1080200070E002C06FEF7FEFC5012DD14C01F32D41
:10803000F0683F2E820133FC19C0822D90E0881633
:108040009906A0F4B60180E290E043D12A94F5CFDE
:10805000F50137FC859137FE81915F01B60190E013
:1080600038D121102A9421E0821A910881149104B8
:1080700079F7E1C0843611F0893639F5F80137FE19
:1080800007C060817181828193810C5F1F4F08C09E
:1080900060817181072E000C880B990B0E5F1F4FBA
:1080A000F32DFF763F2E97FF09C090958095709530
:1080B00061957F4F8F4F9F4FF0683F2E2AE030E051
:1080C000A30143D1882E861844C0853731F4232D6F
:1080D0002F7EB22E2AE030E025C0932D997FB92E55
:1080E0008F36C1F018F4883579F0AEC0803719F0BA
:1080F000883721F0A9C0E92FE061BE2EB4FE0DC083
:10810000FB2DF460BF2E09C034FE0AC0292F266063
:10811000B22E06C028E030E005C020E130E002C009
:1081200020E132E0F801B7FE07C0608171818281F1
:1081300093810C5F1F4F06C06081718180E090E0E9
:108140000E5F1F4FA30101D1882E8618FB2DFF77EC
:108150003F2E36FE0DC0232D2E7FA22E891458F4FB
:1081600034FE0BC032FC09C0832D8E7EA82E05C0C4
:10817000B82CA32C03C0B82C01C0B92CA4FE0FC08E
:10818000FE01E80DF11D8081803321F49A2D997E46
:10819000A92E09C0A2FE06C0B394B39404C08A2DD0
:1081A000867809F0B394A3FC10C0A0FE06C0B214F8
:1081B00080F4280C922C9B180DC0B21458F4B60110
:1081C00080E290E086D0B394F8CFB21418F42B1864
:1081D00002C0982C212CA4FE0FC0B60180E390E0D1
:1081E00078D0A2FE16C0A1FC03C088E790E002C0D0
:1081F00088E590E0B6010CC08A2D867851F0A1FE8A
:1082000002C08BE201C080E2A7FC8DE2B60190E0E3
:1082100060D0891430F4B60180E390E05AD09A948B
:10822000F8CF8A94F301E80DF11D8081B60190E04A
:1082300050D08110F6CF222009F44ECEB60180E254
:1082400090E047D02A94F7CFF6018681978102C04B
:108250008FEF9FEF2B960FB6F894DEBF0FBECDBF0A
:10826000DF91CF911F910F91FF90EF90DF90CF9012
:10827000BF90AF909F908F907F906F905F904F9046
:108280003F902F900895FC010590615070400110BF
:10829000D8F7809590958E0F9F1F0895FC0161502F
:1082A000704001900110D8F7809590958E0F9F1F18
:1082B0000895DC01FC01672F71917723E1F7329774
:1082C00004C07C916D9370836291AE17BF07C8F3B1
:1082D00008950F931F93CF93DF93FB01238121FD1B
:1082E00003C08FEF9FEF2CC022FF16C0468157813D
:1082F000248135814217530744F4A081B1819D0147
:108300002F5F3F4F318320838C93268137812F5FEE
:108310003F4F3783268314C08B01EC01FB0100849F
:10832000F185E02D0995892BE1F6D80116968D91FE
:108330009C911797019617969C938E931697CE0152
:10834000DF91CF911F910F910895FA01AA2728304C
:1083500051F1203181F1E8946F936E7F6E5F7F4F12
:108360008F4F9F4FAF4FB1E03ED0B4E03CD0670F8E
:10837000781F891F9A1FA11D680F791F8A1F911DE1
:10838000A11D6A0F711D811D911DA11D20D009F431
:1083900068943F912AE0269F11243019305D319373
:1083A000DEF6CF010895462F4770405D4193B3E05C
:1083B0000FD0C9F7F6CF462F4F70405D4A3318F003
:1083C000495D31FD4052419302D0A9F7EACFB4E0B4
:1083D000A6959795879577956795BA95C9F700976C
:1083E0006105710508959B01AC010A2E069457950D
:1083F000479537952795BA95C9F7620F731F841F64
:10840000951FA01D0895DC01CB01FC01E199FECF71
:1084100006C0FFBBEEBBE09A31960DB20D92415003
:108420005040B8F70895E199FECF9FBB8EBBE09A0C
:1084300099278DB30895A8E1B0E042E050E0E5CF80
:10844000DC01CB0102C02D9105D041505040D8F73E
:108450000895262FE199FECF9FBB8EBB2DBB0FB693
:10846000F894E29AE19A0FBE01960895F2DF272F61
:06847000F1CFF894FFCFEC
:108476000000000200000000DE0700000000575464
:108486003D2025750A47530047533D2025750A535D
:108496004E00534E3D2025750A454E4400574B3D30
:1084A6002025750A565000503D332E360A5200528A
:1084B6004C3D2025750A68004F3D73740A530047EA
:1084C6003D73740A530053523D53746174696F6E61
:1084D600200A57500057503D536E36332F506233A3
:1084E600370A57540057503D536E41670A57540098
:1084F60057503D50726F66696C65300A5754005785
:10850600503D50726F66696C65310A57540057507A
:108516003D50726F66696C65320A57540057503D7C
:1085260050726F66696C65330A57540057503D5058
:10853600726F66696C65340A57540057503D507225
:108546006F66696C65350A57540053523D5550683D
:108556006561746572200A57500053523D5072652A
:10856600686561746572200A57500053523D4D612B
:108576006E75616C200A57500053523D5265626F0A
:108586006C6C696E67200A57500053523D43686908
:108596007068656174696E67200A57500053523DD2
:1085A60050434268656174696E67200A57500053EC
:1085B600523D5043200A57500056312E310020209C
:1085C60020C2F0E5ECFF20F0E5E1EEEBEBE8EDE3B1
:1085D600E02020202000C2FBE1E5F0E8F2E520F0F3
:1085E600E5E6E8EC00D2E5ECEFE5F0E0F2F3F0E0EA
:1085F60020EFEEEBEEF7EAE8202000EDE8E7E020DA
:10860600EFF0E820E4EEEDE0E3F0E5E2E500D2E5A8
:10861600ECEFE5F0E0F2F3F0E020F3E2E5EBE8F76B
:10862600E5EDE8FF00202020202020E4EEEDE0E349
:10863600F0E5E2E020202020202000C4EBE8F2E56F
:10864600EBFCEDEEF1F2FC20E2EFE8F2FBE2E0ED0E
:10865600E8FF00D4F3EDEAF6E8FF20E4EEEDEEE302
:10866600F0E5E2E000EDE8E6EDE5E3EE20EDE0E33F
:10867600F0E5E2E0F2E5EBFF2020202000CCE0EA86
:10868600F1E8ECE0EBFCEDE0FF20ECEEF9EDEEF1CD
:10869600F2FC202000E2E5F0F5EDE5E3EE20EDE06A
:1086A600E3F0E5E2E0F2E5EBFF20202000CCE0EA93
:1086B600F1E8ECE0EBFCEDE0FF20ECEEF9EDEEF19D
:1086C600F2FC202000E2E5F0F5EDE5E3EE20EDE03A
:1086D600E3F0E5E2E0F2E5EBFF20202000D2E5EC56
:1086E600EFE5F0E0F2F3F0E020E2EAEBFEF7E5ED8D
:1086F600E8FF202000CAEEEDF2F0EEEBFC20EFEEF4
:1087060020E2E5F0F5F320202020202000EDE8E629
:10871600EDE5E3EE20EDE0E3F0E5E2E0F2E5EBFF88
:108726002020202000CAEEFDF4F4E8F6E8E5EDF29C
:1087360020EFF0EEF4E8EBFF2020202000E2E5F049
:10874600F5EDE5E3EE20EDE0E3F0E5E2E0F2E5EB62
:10875600FF20202000CAEEFDF4F4E8F6E8E5EDF28D
:1087660020EFF0EEF4E8EBFF2020202000EDE0E320
:10877600F0E5E2E0F2E5EBFF202000D2E5ECEFE5E4
:10878600F0E0F2F3F0E020EDE8E6EDE5E3EE2020A0
:10879600202000EFE0E9EAE82000D2E5ECEFE5F082
:1087A600E0F2F3F0E020ECE5F1F2E02020202020DA
:1087B60000C2FBE1E5F0E8F2E520EFF0EEF4E8EBCD
:1087C600FC00CFF0EEF4E8EBFC203500CFF0EEF441
:1087D600E8EBFC203400CFF0EEF4E8EBFC203300AD
:1087E600CFF0EEF4E8EBFC203200CFF0EEF4E8EB4D
:1087F600FC203100CFF0EEF4E8EBFC203000536EA5
:10880600416700536E506200CAEEECEFFCFEF2E5E3
:10881600F000C4EEEF2E20EDE0F1F2F0EEE9EAE82A
:1088260000EFEBE0F20020D1F3F8EAE020EFEBE016
:10883600F22000ECE8EAF0EEF1F5E5EC00D1F3F811
:10884600EAE000D0E5E1EEEBEBE8EDE32000D0F363
:10885600F7EDEEE9002020D0F3F7EDEEE920202039
:1088660000CDE8E6EDE8E920EDE0E3F02E2000C2D9
:10887600E5F0F5EDE8E920EDE0E3F02E002020D16B
:10888600F2E0EDF6E8FF00E2E5F0F5E000EDE8E7FE
:10889600E000CCEEF9EDEEF1F2FC00CFF0E8EDFFF2
:1088A600F2EE202000C2DBC1D0C0D2DC00C2DBCA9F
:1088B600CB00C2CACB00CDE0F1F2F0EEE8F2FC004C
:1088C600C7E2F3EAEEE2FBE520F1E8E3EDE0EBFBDD
:1088D60000CFF0E5E4F3F1F2E0EDEEE2EAE800D3F2
:1088E600ECEEEBF7E0EDE8FF00C2F0E5ECFF20EF81
:1088F600E0E9EAE80020C4E0F2F7E8EA20EDE8E67D
:108906002E20EDE0E3F0E5E2E0F2E5EBFF0020C427
:10891600E0F2F7E8EA20ECE5F1F2E020EFE0E9EA40
:10892600E800F0F3F7EDEEE900EDE8E6EDE8E90042
:10893600EDE0E3F02E00C2E5F0F5EDE8E900C2DB7C
:04894600D5CEC400C6
:00000001FF
